:020000040000FA
:100000000250040001000000900400009004000071
:100010009004000090040000900400009004000090
:100020009004000090040000900400009004000080
:10003000900400006A510000900400009004000049
:100040009004000090040000900400009004000060
:100050009004000090040000900400009004000050
:100060009004000090040000900400009004000040
:10007000900400009E5200009004000090040000D4
:100080009004000090040000900400009004000020
:1000900090040000AC510000C85100009004000022
:1000A0009004000090040000900400009004000000
:1000B00090040000900400009004000090040000F0
:1000C00090040000900400009004000090040000E0
:1000D00090040000900400009004000090040000D0
:1000E00090040000900400009004000090040000C0
:1000F00090040000900400009004000090040000B0
:10010000900400009004000090040000900400009F
:1001100090040000900400000044000090040000DF
:10012000900400009004000090040000900400007F
:10013000900400009004000090040000900400006F
:10014000900400009004000090040000900400005F
:10015000900400009004000090040000900400004F
:10016000900400009004000090040000900400003F
:10017000900400009004000090040000900400002F
:10018000900400009004000090040000900400001F
:10019000900400009004000090040000900400000F
:1001A00090040000900400009004000090040000FF
:1001B00090040000900400009004000090040000EF
:1001C00090040000900400009004000090040000DF
:1001D00090040000900400009004000090040000CF
:1001E00090040000900400009004000090040000BF
:1001F00090040000900400009004000090040000AF
:10020000FFFFFF00FFFFFF009004000090040000CC
:10021000900400009004000090040000900400008E
:10022000900400009004000090040000900400007E
:10023000900400006A510000900400009004000047
:10024000900400009004000090040000900400005E
:10025000900400009004000090040000900400004E
:10026000900400009004000090040000900400003E
:10027000900400009E5200009004000090040000D2
:10028000900400009004000090040000900400001E
:1002900090040000AC510000C85100009004000020
:1002A00090040000900400009004000090040000FE
:1002B00090040000900400009004000090040000EE
:1002C00090040000900400009004000090040000DE
:1002D00090040000900400009004000090040000CE
:1002E00090040000900400009004000090040000BE
:1002F00090040000900400009004000090040000AE
:10030000900400009004000090040000900400009D
:1003100090040000900400000044000090040000DD
:10032000900400009004000090040000900400007D
:10033000900400009004000090040000900400006D
:10034000900400009004000090040000900400005D
:10035000900400009004000090040000900400004D
:100800000FB421000EDF23000E018800000000005D
:100810000C000700606F2400010020001100070099
:10082000000020000000E000020032000000020092
:1008300000000000903D0200000000000040DA00CF
:100840000000FE004440A900E05521000000E00047
:100850000300320000002000A00188004440A800EE
:100860000000060091018800800078000000EB0085
:1008700015003700E280400032A0B4009101BA00B8
:10088000E280400032A0B4009102BA00E280400051
:1008900032A0B4000002EB00472BDE00F507B200E7
:1008A000602CE10004003A000059EB008301E900EC
:1008B000FDFF3E00040037006128E1000100320026
:1008C0000082EB00040007001101BA000200E00002
:1008D000E8FF3A00000006003159BA008301E90040
:1008E0000C0032002159BA008301E90008003200EF
:1008F0000400E00003003A00E280400032A0B400AF
:10090000F5FF370011D9BA008301E900FAFF3A0078
:100910008100E800E180400032A0B4000000060041
:100920000040DA000000FE000A00FA0080017800B2
:10093000E20F500028003E00B03F8200E10F50005F
:1009400008003200802320000000E0000500320093
:100950000423200025232000462320008001780066
:100960000400370004222000252220004622200017
:1009700083222000144090000004E00004003500B1
:100980008009EB00144090000074A0001042980011
:10099000154090000028A30003003A001540900085
:1009A0000024A000904298008001EB00070037006F
:1009B000154090000008A300FDFF320063C07800DE
:1009C0000000FB00000B78008301E800828F5100DB
:1009D000F7FF3A000800370030002000B0BF9F004A
:1009E000C3BF9F00D1BF9F00E2BF9F006A80570036
:1009F00000C0DA006FB99700020078000080FA00AA
:100A000000000600889FBE008A9FBE000105780096
:100A10000100E0000400350008003C000000E00098
:100A2000200032000500370060001000E080180050
:100A300002003B0001F02C001A0037000004BE0049
:100A40006011B8006B0920000982CF000200390054
:100A50000882CF000441B000694252000E0032000B
:100A600008003B0082817100610164008904D100AB
:100A70000884D3008B05E8000442E800F9FF3A003F
:100A8000050037000804440089844C008B05E90008
:100A90000442E900FBFF3A00720107000AF0A700D8
:100AA00001F0A0004F05BE004F04BE00000006008C
:100AB00003F0A200889FBE008A9FBE008C1F7800B2
:100AC0008E010700950133006450E1004F003200B1
:100AD0006420E1005200320003826C0007003B00FA
:100AE0000905D0000306D000820F54000C065D00FB
:100AF0000200390002003200890178000306780004
:100B00008582550004003D000003FD008103FD00C7
:100B10008502EA008B854200840F720002003B00D0
:100B200060001000E08018006011B8000005EB00C4
:100B30007A28E1000A00390006007800C75DDD0070
:100B4000F707B200878075002D00370082817100A1
:100B50000A017800610560008180D1000080D30027
:100B60008502E900F9FF3B00060440008784480045
:100B700002003B0060041400E0841C000988A3000C
:100B8000070032008A817100828171006101640076
:100B90008904D1000884D3008B05E80017003700D2
:100BA0000978A30013003A000B00E00013003400A2
:100BB0008B05E9000804440089844C000A44740051
:100BC0000978A3000D003A000B00E0000700340094
:100BD0008B05E9000804440089844C0001003A00B8
:100BE0000B0020000978A300F7FF32000001EB00A2
:100BF00002003700828171000A01780019010700A4
:100C00000CF0A70001F0A0004D0137006420E100C6
:100C100002003A00838F6C004D0133000801BE00D2
:100C20000200BE0046013700889FBE008A9FBE00BA
:100C30008C1F7800310107003801330003866C00F7
:100C40006450E100240032006420E10027003200FB
:100C50006150E100220032006120E10021003200F9
:100C60008B854200EB07B1000134B800003AB800B0
:100C70000804420089844A00013AB8000030B800F4
:100C80008880400009014A00040033000000400051
:100C900081804800020149008B05E900C909DD0097
:100CA000830170000100320013002000C814DE0030
:100CB0004814DD004709DE001200B200C808DE005B
:100CC00008847000E700070001F0A1000CF0A70005
:100CD00001F0A0001A0137006120E1001C01320080
:100CE0000801BE000200BE00F7FF37006150E100BE
:100CF000FCFF3A00160137000001BE001701070093
:100D00000470A70003F0A10003F8A30013003A0049
:100D10006509B10010003200090035006928E100C2
:100D2000020035000100280000000500000040001E
:100D3000818048008502E900FCFF3A0000000600BF
:100D4000F88F4200050035008100D1000080D300FB
:100D50008502E800FCFF3A00000006008000EB007E
:100D600000000500889FBE008A9FBE008C1F78008F
:100D7000E2000700E900330003866C006450E100E4
:100D80002E0032006420E100330032006150E100A7
:100D90002F0032006120E1003100320085855500CE
:100DA000EB07B00009002000080420000500370010
:100DB0000804440089844C000A0031000603430003
:100DC00087834B000001530081815B00F8FF3300F3
:100DD0000203BE000800A0000804440089844C00FF
:100DE000F6FF3900C639DD008301730001003200CF
:100DF000130020008904D1000884D3000998A300BF
:100E0000050032000800A7000300A0008904D100FB
:100E10000884D3008B05E8008904D1000884D3003E
:100E20000001EB000281D2008E00070001F0A1005A
:100E30000CF0A70001F0A000C10037006420E10021
:100E4000C30032000801BE000200BE00F7FF3700F9
:100E50006120E100BE0032006000B800F3FF3700FF
:100E60000000200001F82700F0FF3700889FBE0037
:100E70008A9FBE008C9FBE00CD00070085047800CD
:100E80000005BE006420E10049003E006220E10050
:100E900003003200090035000BF8A30044003200C3
:100EA0000BF8A3000800320010022000F0D98800DF
:100EB000F0FF2F00F1FF27003D00370001F82F0061
:100EC000000020003A0037003D000700F8FE070050
:100ED0000006BE000A00BE00324F200053F323007C
:100EE0005E000700060034000C00BE00340007005E
:100EF000EFFE07000006BE000A00BE000200370039
:100F00008904E9000C00BE002D00070046FF070021
:100F10002B000700E7FE07000001BE000C00BE002A
:100F200090FF07000005BE000001BE003EFF070065
:100F30000006BE00A2F32300430D2C00DDFE0700D7
:100F4000809FBE000C00BE00D2E32700D3F02B0030
:100F500035FF07004F01BE0082FF07000006BE00FC
:100F60000A01BE0030FF07000A01BE00D1FE0700E3
:100F70000006BE006148B900A2FE07000005BE00E1
:100F800032082800E3952B0027FF07000C01BE0064
:100F9000C8FE07000006BE000A00BE0002002800CE
:100FA00013F3230020FF07000C01BE00C1FE070061
:100FB0004F06BE004F05BE004F04BE0000000600F5
:100FC00003F02300020005000001BE0063000700DB
:100FD0000470A70003F0A1006509B10016003200FB
:100FE0000D0035006828E10006003500F0FF2F00F5
:100FF000F1FF27000300E00013003B000100280080
:101000000000050000004000818048008502E900E2
:10101000FCFF3A0008003700F88F420002003C0055
:101020008000EB00000005008100D1000080D300AB
:101030008502E800FCFF3A000300E00002003B00EC
:1010400060001000E08018000000060087FF070025
:1010500092BD2500E3ED2300F3FE3700F4FF2F00DF
:101060006000370081002000618055000B003D00CA
:101070000B00200061FE2F000100E1001D00340084
:1010800082817100610164008904D1000884D30069
:101090000000E800FAFF3A007100200061006400DF
:1010A0000300700002006000090032006104440087
:1010B000E0844C000988A500050032008B05E8009B
:1010C0006808E10002003A008904D1000884D300D6
:1010D000F20F20000258E10005003D00C75DDD0071
:1010E000F907B2008980750008007800000006004A
:1010F0000BF827008B007800000005000004BE00FC
:10110000160007000003BE000405BE000200BE007A
:1011100012000700844F7500000006000200BE00A8
:101120006450E100050036006420E1000200360052
:101130000968A30001003A000800BE000160A00099
:101140004F0678004F05BE004F04BE0000000600A9
:10115000F0FF2F00F1FF2700F9FF3700C70ADE007C
:10116000F107B200F50FB20008003200E1CF4200F3
:10117000020032000170A00024000500810F700001
:10118000010032000408050044000500810F7000D2
:1011900002003A00140005008502E900000040004A
:1011A00081C04800FCFF3B000170A0002400050046
:1011B0000003BE00E9FF07006220E10002003200E8
:1011C0000600BE0005000500E507B100F107B2000A
:1011D00004F023008480700007F0A70001F0A00055
:1011E00024000500889FBE008A9FBE00841F7800EF
:1011F000C2FF07004F00780011003300F0FF2F00FE
:10120000838F6C0006003B00040565000A00A70000
:101210000800370009F0A600100020000800370081
:10122000820F5400838F5C000300390010002000FF
:1012300001003E000000200009F0A7000000EA00C5
:101240004F05BE004F04BE000000E0000000060095
:10125000881F7800000478005001BE004000BE00E6
:10126000040040008580480006014900878149004C
:10127000009CBE000294BE000400E1000588E1006D
:101280000690E1000798E100020031006800440088
:101290001008E8004F04780000000600F4874700BB
:1012A000889FBE008A9FBE008C9FBE008E1F780064
:1012B0000205BE000004BE00D4B79F00E5B79F0042
:1012C000F6B79F0087BF9F000000EB00C0B79F00EC
:1012D000B0B79F00A0B79F0090B79F0080B79F0056
:1012E0000D042000BFB097004FB0970000014000F0
:1012F0000000E0000F003D004F08DE00000071001C
:10130000C0B79F009E00070001003D0012002000B2
:10131000A100070001003D0012002000A600070008
:10132000B1000700B60007000F004000C8FF07002B
:10133000220037004F08DE0000067100CCB79F0086
:101340008F00070001003D001200200092000700FE
:1013500001003D001200200097000700A2000700D6
:101360000FB297009FB297002FB39700BFB39700BB
:10137000A90007000000520081805A0002015B00B2
:1013800083815B0080B79F0091B79F00A2B79F0049
:10139000B3B79F000007EB009F0007000020E100AB
:1013A00001A8E10002B0E10003B8E1000100310052
:1013B0001E0020000E005600C0B79F004FB29700DD
:1013C0000400E000070035001000200001002000AC
:1013D0006011B80008047000898470000A0571006B
:1013E0008B8571008D06E900BEFF3A000400E00025
:1013F00003003D00820007000F00400094FF07003B
:101400004FA897000000E00004003A000FB49700D6
:101410009FB497002FB59700BFB5970094000700C1
:101420004F0778004F06BE004F05BE004F04BE00B8
:101430004F01B10000000600881F7800180020004E
:10144000881F780095FF07008F87E9004F04780018
:1014500000000600801FEB0090FF07008F87E90067
:1014600000000600889FBE008A9FBE008C1F780087
:101470006E00070007003D0073000700E00F5B00EF
:10148000E08F5B0007003D00320007000006EB0024
:10149000040037003400070002003D002A00070066
:1014A0001C00200072000700E3FF07000203BE00DB
:1014B0000002BE000C00E000010032002200070024
:1014C0000400BE000601BE004F0678004F05BE00B6
:1014D0004F04BE0000000600889FBE008A9FBE0029
:1014E0008C1F78005100070005003D0056000700E2
:1014F000E00F5B00E08F5B0006003D00040037005A
:101500001900070003003D006000B8006011B8003A
:101510001000070056000700CEFF07000203BE00C0
:101520000002BE000C00E0000100320006000700CF
:101530000400BE000601BE004F0678004F05BE0045
:101540004F04BE00000006006000B8006011B80043
:10155000000037000402500085825800060359003D
:1015600087835900000006000006EB00E00F5200E0
:10157000E08F5A00E00F5B00E08F5B000000060088
:101580000180400090B79F000001EB008FB09700F2
:101590000100E000000006000200700090B79F000C
:1015A0000180400080B79F000001EB00FFA897007A
:1015B0000100E000000006000200700080B79F00FC
:1015C000018040006FAA9700CF20DE00010070006C
:1015D000F0AF9F0004024200250007004F18DE0014
:1015E0000002720000000600E4AF9F0008044400FF
:1015F00089844C000A054D008B854D0000000600D3
:101600003FB29700CFB297005FB39700EFB3970058
:1016100000FE2F00000006003FB09700CFB09700FB
:101620005FB19700EFB19700000006000205BE0011
:101630000004BE00E00F5000E08F5800E00F59009A
:10164000E08F5900000006006000B8006011B8008B
:1016500008045000898458000A0559008B855900F8
:101660001C002000E00F5200E08F5A00000006002E
:101670000800BE000A01BE0000000600889FBE00F0
:101680008A9FBE008C9FBE004400F800070F200018
:10169000270288003400F80007F02F000338E1002B
:1016A00004003200270280004700B30027028800B0
:1016B000A3018800811F780019002000804CDD0004
:1016C0001300200002047800800678008904D1000D
:1016D000424EDD00010578000302E90004800800A5
:1016E000170000008A0546004218DD000902E900E3
:1016F0000480080010000000000000004620C30025
:101700003B025200DF35C100080440001381C200D3
:10171000AB825200264DC5003E85C400BB00CD0003
:10172000BB80CD003A00CA002A80CA000700C90069
:101730000580C900BA00CD00BA80CD000A05460078
:10174000020478008301D0008D06E900DFFF3C0031
:101750004F0078003400F9004400F9004F06BE0045
:101760004F05BE004F04BE00000006004600F80012
:101770005000F800022020003202880002002800F9
:10178000130020008019DD000281710082028800B0
:1017900001007800010178002600200047002000A9
:1017A0008301E90003800800070000000110E10048
:1017B000040034001102BE0092087800E2307B0081
:1017C0000489BE0087804000121978005000F9009B
:1017D0004600F900000006000C00FA00889FBE00D9
:1017E00000047800CFB09700F0FF2700D0BF9F0023
:1017F0008004EB0099BF9F0088BF9F00A8BF9F0097
:10180000200C2000B0BF9F007881570070805700E7
:10181000140007000FB89700094878000FB8970028
:1018200008045000080078004F04BE000080FA0051
:1018300000000600800178000001780001003700F8
:101840000201E8001204E000FDFF3A003140780098
:10185000005978000004E000FCFF3A000300780023
:1018600000000600FE874700889FBE008A9FBE00DA
:101870008C9FBE008E1F7800F0B79F000107780094
:1018800082BF9F000000EB00A0B79F009F023700BF
:101890008006EB0050C2B30080CF50000900320038
:1018A0000100FB00FFB09700A3020700E10F40001A
:1018B00096023200AFB097008100E800A1B79F0008
:1018C000920237009E407800D0C2B30080CF500013
:1018D0000C00320007003C006D40500080CF5000EB
:1018E0000A0032006B40400080CF50000E003A00EA
:1018F0000800370000C3B30080CF50000A003A0050
:10190000060037000D30A000050037000D00A000D4
:10191000030037000D10A000010037000D20A000CB
:101920000E07E800E7FF37000D18A30001003200A2
:101930000D00A1000D38A300010032000D20A10010
:101940000100FB0002FD2F0002004000E90F5000E3
:101950000E003E000002EB00C4B79F008201780039
:10196000CFB297006A28B9001E01FB0000014100B8
:1019700003014100C2B79F005E00FB00030040006E
:10198000E90F50000B003E00F5FF37000006EB00AA
:10199000CCB79F00A0C2B30080CF500005003A0032
:1019A0000FB89700C000780080BF9F00C1B79F00AC
:1019B0000E07E8000001EB00B2B79F00E0C2B300E1
:1019C0009E4F100018003A000DE0A0008E00E800C5
:1019D00064405000914F100002003200010778006F
:1019E0000C0037000FBA9700C402780084BF9F0034
:1019F000B5B79F000E87E8000B0037003FB6970091
:101A00006A60B9000000410003004000B0B79F00C9
:101A10000E07E8001E01FB0003FD2F00030041003C
:101A2000E90F5000F5FF3600BE407800E1D79F0077
:101A3000C0C6B30080CF5000220032000F003C002F
:101A40006940500080CF50007700320004003C0015
:101A50000104E000310232006B4050000F003700FB
:101A600040C6B30080CF5000930032006540400074
:101A700080CF50008B003A008F00370030C7B30092
:101A800080CF50001A00320007003C006440500034
:101A900080CF5000110032000040E80080CF50009D
:101AA00080003A000F00370050C7B30080CF5000CD
:101AB000800032006340400080CF500079003A003F
:101AC00009003700000028000D48A30001003A007B
:101AD0000001200080867600D3FF37000D60A00053
:101AE000750037000D50A0000D70A0007200370087
:101AF0008FB897004100780081BF9F0000047800F4
:101B00000000E00001003A00087A24008004EB00A5
:101B1000010037008104E800890078000880440053
:101B20001004E000FBFF3A003FB197000200E00024
:101B300003003200890F5100010031008204780057
:101B40000002EB00E4AF9F00CFB29700898F5200F4
:101B50000200360009805200E0AF9F004368DE00BB
:101B6000E10660001B003A000D067800090037000E
:101B7000FFB0970000022000EF010700E10F4000D6
:101B8000030032002FB097000000E800A0B79F00CC
:101B90000C06E800EFA89700810F5600F4FF3A000A
:101BA0000081EB00E2AF9F000A0037008800780058
:101BB0003100FB0001047800FFB09700DE01070050
:101BC000E10F4000030032002FB297000402E8004A
:101BD000A4B79F000900E90080047800E10F4000ED
:101BE000F2FF3A000006EB000D00E0000A003A00A8
:101BF000C6013700FFB0970000022000CE010700A9
:101C0000E10F400003003200AFB297008502E80008
:101C1000A5B79F000C06E8006FA89700800F56003C
:101C2000F4FF3A00B90137008FB8970041007800FF
:101C300081BF9F00CF80DE00010178008201780023
:101C40000205BE000004BE000203BE000002BE008A
:101C50004822DE00482EDD0004027600E4D79F0013
:101C60000D48A3000A0032000404E000080032001E
:101C7000E14F42000600320071FD2F000180470055
:101C8000044878001840980029002000020037001E
:101C9000F0D79F001900200072FD2F00028447003A
:101CA000A1FF370064FD2F000484470019002000C5
:101CB0009DFF37000D0CB3000D007800000CB20042
:101CC00028003A000D00E00005003D008FBA9700A3
:101CD0004505BE004504BE0085BF9F0014003700C7
:101CE0000D48A3000B0032000FBE97004C00BE0051
:101CF0008CBF9F004F89DE00CF91DE000002BE0046
:101D000002037800820378000605BE000404BE00CA
:101D1000070037008FB897004100780081BF9F000F
:101D200000047800CFC4DE00090578008A05780039
:101D3000E00F5400E08F5C00E00F5D00E08F5D007D
:101D40001F003D003D00B3006000B8006011B80006
:101D500008045000898458000A0559008B855900F1
:101D6000170037000D00E00005003D000FB9970097
:101D70004205BE004204BE0082BF9F001000370033
:101D80000D48A300070032000FBA97004400BE00C0
:101D900084BF9F006011B8000205BE000004BE00B1
:101DA000070037008FBA97004500780085BF9F0075
:101DB00000047800090020000A0020000B00200029
:101DC0003FB697000C00E00007003A00E00F540017
:101DD000E08F5C00E00F5D00E08F5D0002003A00E4
:101DE00010002000B0B79F008D007800010CB200F9
:101DF000E1B79F0000042000808F500030003200C7
:101E000003003C000100E000080032004000370001
:101E1000000820006FB19700800F510014003200BD
:101E2000000C2000800F510039003A0014C0B300AC
:101E3000057024000B0037000400FB004300DD00A8
:101E4000050040005001BE004000BE000040E1001F
:101E500001C8E10002D0E10003D8E1002B00390005
:101E60000442E800F44F5200F3FF3A002700370025
:101E700000012000010020006011B80014C0B30070
:101E80000040E10001C8E10002D0E10003D8E10018
:101E90001E003900450020000000D0008180D200E3
:101EA0000281D2008381D2008502E900FAFF3A0064
:101EB0000442E800F04F5200F1FF3A0013003700EF
:101EC00080002000010020006011B80014C0B300A1
:101ED0000040E10001C8E10002D0E10003D8E100C8
:101EE0000A0039003C0020000000D0008180D200B0
:101EF0000281D2008381D2000C06E900FAFF3A0089
:101F00000442E800F54F5200F1FF3A00E4D79F0089
:101F1000EFD097000100FB003FB19700820F500007
:101F200002003D00E2D79F00040037003FB2970057
:101F3000800F520001003D00B0B79F00CFB2970064
:101F40000500E000040032006380660002003200F9
:101F50008502E900C5B79F000DE8A3000B00320021
:101F60004FB697003FB09700800F560003003C002B
:101F70008000EB00C1B79F00040037004FB197000D
:101F80003FB2970004015100C2B79F00EFD2970003
:101F90000500FB000006EB00DCAF9F00CFB0970010
:101FA000808F50000200340000805000D0AF9F00AE
:101FB0000D28A30037003200E18066000D18A30051
:101FC0000C003200D00220000100E00001003A00C5
:101FD0000080E900FFB09700D7000700E10F400044
:101FE0000E0032002FB197000201E800A2B79F0057
:101FF0000A0037000100E00008003200FFB097003F
:1020000000022000CC000700E10F40000300320076
:102010002FB297000402E800A4B79F00DFAA970040
:102020000500E0000F0032000006EB00FFB0970053
:1020300000032000C0000700E10F40000300320051
:102040002FB097000000E800A0B79F000C06E80042
:10205000DFA89700810F5600F4FF3A000001EB0063
:10206000D2AF9F003FB29700C320DD00806F2400F5
:102070008080400091B79F004220DD006400500046
:1020800080B79F006320B900F0AF9F006306500047
:1020900084003700DFAA97000500E000110032003D
:1020A000688066000F003A0000067800FFB09700D5
:1020B00000022000A0000700E10F400003003200F2
:1020C0002FB097000000E800A0B79F000C06E800C2
:1020D000DFA89700810F5600F4FF3A000001EB00E3
:1020E000D2AF9F00E18066000D18A3000C00320003
:1020F000D00220000100E00001003A000080E90069
:10210000FFB097008C000700E10F4000D5FF3200C0
:102110002FB297000402E800A4B79F00D1FF370058
:102120000100E000CFFF3200FFB097000002200066
:1021300081000700E10F4000CAFF3200AFB29700F4
:102140008502E800A5B79F00C6FF37000004200005
:10215000EFB09700808F50003100320003003C0048
:102160000100E000080032003E00370000082000B7
:102170006FB19700800F510011003200000C200059
:10218000800F510037003A001FB097003002BE00A8
:102190002003BE000800BE000A01BE00A6FC070026
:1021A000A4002000050020006033B800A9FC07004F
:1021B00004C3B30004424000E4D79F002900370065
:1021C000757A2400D5B79F000D58A30002003A008D
:1021D000807B2400D0B79F00140020000500200061
:1021E0006033B8008FB097008100E900050033002C
:1021F0000402D0008582D2000683D2008783D200F9
:10220000F9FF37000800BE000A01BE008AFC070083
:102210006F0060005FB197006240780010003700E7
:1022200014002000050020006033B8000C00780086
:102230000000E900050033000402D0008582D200CE
:102240000683D2008783D200F9FF37000800BE0062
:102250000A01BE0078FC0700674060000043B00040
:10226000E0D79F00EFD097000100FB00FFB0970080
:1022700031000700E10F4000030032002FB197004A
:102280000201E800A2B79F001FB297006802520047
:1022900094B79F008FB29700E482520085B79F00E9
:1022A00063065600D0FF2F003FB197000090B900A1
:1022B0007FAA97000000420063005000800F560084
:1022C000A2FF3A000D38A30010003200DFAA9700E9
:1022D0000500E0000D0034000006EB00FFB09700A1
:1022E0000002200014000700E10F4000030032004C
:1022F0002FB097000000E800A0B79F000C06E80090
:10230000DFA89700810F5600F4FF3A00BE40780026
:10231000E1D79F000104E0005DFD3A002FB0970077
:102320004F0778004F06BE004F05BE004F04BE00A9
:10233000EF01B10000000600889FBE000001780098
:1023400001047800B10090000118A3003D003200A4
:102350000198A30003003A00180090000000E0007C
:1023600038003A000190A0003104980082047800FF
:10237000F90FB200180090000000E00002003A00DF
:1023800028009000000C7800EA8F540006003A0004
:10239000380090000078A30003003A00880078001D
:1023A000D0002000E4FF0700980090005800900043
:1023B000808F50000B0032000100E80010049800EC
:1023C0001800780009587800000C780011C0B3009C
:1023D000407F240001487800EA8F54000600320054
:1023E00019003700880078000940780019000700BC
:1023F0008004780014003700380090000088A300A3
:102400001100320018019000A800900048009000D0
:1024100045F9070098009000810F50000400320039
:10242000380090000003B300300498008084EB0073
:102430000000EB001004980028009000000C7800C9
:10244000010037008084EB00090078004F04BE00D3
:10245000000006000200FA00889FBE00A0FF9F0057
:1024600001047800B1009000810478000904B200F2
:10247000020032000000FB00360037000118A30004
:1024800005003A000103B3003104980019049800D4
:102490000080EB002F003700580090000000E000A3
:1024A00006003A004800900012002000E680570025
:1024B0001DF9070019049800240037002800900037
:1024C0000000E00008003A00007F2400200498008B
:1024D000000C7800200020005004980010049800A0
:1024E0000130A0003104980018019000A80090006D
:1024F000480090000CF9070028009000000C7800BC
:102500000080EB001004980018007800AFF89700E6
:1025100001587800000C78002FF89700EA4F50001F
:102520000A003A00380090000088A300070032003B
:1025300018019000A800900048009000FAF80700E9
:1025400019049800A8009000010C7800AFF89700DB
:102550000100FB004F04BE000080FA0000000600EE
:10256000000000003200000064000000960000003F
:10257000C9000000FB0000002D0100005F01000009
:1025800092010000C4010000F601000028020000D2
:102590005B0200008D020000BF020000F10200009B
:1025A000240300005603000088030000BA03000063
:1025B000ED0300001F04000051040000830400002C
:1025C000B6040000E80400001A0500004C050000F5
:1025D0007E050000B1050000E305000015060000BF
:1025E000470600007A060000AC060000DE06000088
:1025F000100700004207000074070000A707000052
:10260000D90700000B0800003D0800006F0800001B
:10261000A1080000D40800000609000038090000E5
:102620006A0900009C090000CE090000000A0000B1
:10263000320A0000650A0000970A0000C90A00007B
:10264000FB0A00002D0B00005F0B0000910B000047
:10265000C30B0000F50B0000270C0000590C000014
:102660008B0C0000BD0C0000EF0C0000210D0000E1
:10267000530D0000850D0000B70D0000E90D0000AE
:102680001B0E00004D0E00007F0E0000B10E00007A
:10269000E30E0000150F0000470F0000790F000047
:1026A000AB0F0000DC0F00000E1000004010000017
:1026B00072100000A4100000D610000007110000E6
:1026C000391100006B1100009D110000CF110000B6
:1026D0000012000032120000641200009612000086
:1026E000C7120000F91200002B1300005D13000058
:1026F0008E130000C0130000F2130000231400002A
:102700005514000086140000B8140000EA140000FC
:102710001B1500004D1500007E150000B0150000CF
:10272000E1150000131600004416000076160000A4
:10273000A7160000D91600000A1700003C17000079
:102740006D1700009F170000D0170000011800004F
:10275000331800006418000095180000C718000026
:10276000F8180000291900005B1900008C190000FE
:10277000BD190000EE190000201A0000511A0000D7
:10278000821A0000B31A0000E41A0000151B0000B2
:10279000461B0000781B0000A91B0000DA1B00008C
:1027A0000B1C00003C1C00006D1C00009E1C000067
:1027B000CF1C0000001D0000311D0000621D000044
:1027C000931D0000C31D0000F41D0000251E000025
:1027D000561E0000871E0000B81E0000E81E000004
:1027E000191F00004A1F00007B1F0000AB1F0000E4
:1027F000DC1F00000D2000003D2000006E200000C6
:102800009F200000CF2000000021000030210000A8
:102810006121000091210000C2210000F22100008E
:10282000232200005322000084220000B422000072
:10283000E42200001523000045230000752300005A
:10284000A6230000D6230000062400003624000042
:102850006724000097240000C7240000F72400002C
:10286000272500005725000087250000B725000018
:10287000E725000017260000472600007726000005
:10288000A7260000D72600000727000037270000F2
:102890006727000097270000C6270000F6270000E2
:1028A000262800005628000085280000B5280000D2
:1028B000E5280000142900004429000073290000C5
:1028C000A3290000D2290000022A0000312A0000BA
:1028D000612A0000902A0000C02A0000EF2A0000B0
:1028E0001E2B00004E2B00007D2B0000AC2B0000A7
:1028F000DB2B00000B2C00003A2C0000692C0000A0
:10290000982C0000C72C0000F62C0000252D00009C
:10291000542D0000832D0000B22D0000E12D000099
:10292000102E00003F2E00006E2E00009D2E000095
:10293000CC2E0000FA2E0000292F0000582F000096
:10294000862F0000B52F0000E42F00001230000099
:10295000413000006F3000009E300000CC3000009D
:10296000FB300000293100005831000086310000A2
:10297000B4310000E3310000113200003F320000AA
:102980006D3200009C320000CA320000F8320000B4
:10299000263300005433000082330000B0330000BF
:1029A000DE3300000C3400003A34000068340000CC
:1029B00096340000C3340000F13400001F350000DD
:1029C0004D3500007A350000A8350000D6350000EE
:1029D00003360000313600005E3600008C36000001
:1029E000B9360000E7360000143700004137000018
:1029F0006F3700009C370000C9370000F637000031
:102A000024380000513800007E380000AB38000048
:102A1000D838000005390000323900005F39000065
:102A20008C390000B9390000E6390000123A000084
:102A30003F3A00006C3A0000993A0000C53A0000A5
:102A4000F23A00001F3B00004B3B0000783B0000C7
:102A5000A43B0000D13B0000FD3B0000293C0000EE
:102A6000563C0000823C0000AE3C0000DB3C000015
:102A7000073D0000333D00005F3D00008B3D00003E
:102A8000B73D0000E33D00000F3E00003B3E00006C
:102A9000673E0000933E0000BF3E0000EB3E00009A
:102AA000163F0000423F00006E3F0000993F0000CB
:102AB000C53F0000F03F00001C4000004740000000
:102AC000734000009E400000CA400000F540000036
:102AD000204100004C41000077410000A24100006D
:102AE000CD410000F8410000234200004E420000AA
:102AF00079420000A4420000CF420000FA420000E8
:102B000025430000504300007A430000A543000025
:102B1000D0430000FA430000254400004F44000069
:102B20007A440000A4440000CF440000F9440000AF
:102B3000234500004E45000078450000A2450000F6
:102B4000CC450000F6450000204600004A46000043
:102B5000744600009E460000C8460000F246000091
:102B60001C470000464700006F47000099470000DF
:102B7000C3470000EC470000164800003F48000033
:102B80006948000092480000BC480000E548000089
:102B90000E49000038490000614900008A490000E0
:102BA000B3490000DC490000054A00002E4A00003D
:102BB000574A0000804A0000A94A0000D24A00009B
:102BC000FA4A0000234B00004C4B0000744B0000FD
:102BD0009D4B0000C54B0000EE4B0000164C000062
:102BE0003F4C0000674C00008F4C0000B84C0000C8
:102BF000E04C0000084D0000304D0000584D000032
:102C0000804D0000A84D0000D04D0000F84D0000A0
:102C1000204E0000484E00006F4E0000974E00000E
:102C2000BF4E0000E64E00000E4F0000354F000082
:102C30005D4F0000844F0000AC4F0000D34F0000F8
:102C4000FA4F000021500000495000007050000071
:102C500097500000BE500000E55000000C510000ED
:102C6000335100005951000080510000A75100006D
:102C7000CE510000F45100001B52000041520000F0
:102C8000685200008E520000B5520000DB52000076
:102C900001530000285300004E53000074530000FD
:102CA0009A530000C0530000E65300000C5400008B
:102CB00032540000585400007D540000A35400001A
:102CC000C9540000EF540000145500003A550000AC
:102CD0005F55000085550000AA550000CF55000043
:102CE000F45500001A5600003F56000064560000DC
:102CF00089560000AE560000D3560000F85600007A
:102D00001D57000042570000665700008B57000017
:102D1000B0570000D4570000F95700001D580000BC
:102D200042580000665800008A580000AF58000062
:102D3000D3580000F75800001B5900003F5900000D
:102D40006359000087590000AB590000CF590000BB
:102D5000F3590000165A00003A5A00005E5A00006B
:102D6000815A0000A55A0000C85A0000EC5A000021
:102D70000F5B0000325B0000565B0000795B0000D7
:102D80009C5B0000BF5B0000E25B0000055C000094
:102D9000285C00004B5C00006D5C0000905C000053
:102DA000B35C0000D65C0000F85C00001B5D000016
:102DB0003D5D00005F5D0000825D0000A45D0000DD
:102DC000C65D0000E95D00000B5E00002D5E0000A6
:102DD0004F5E0000715E0000935E0000B45E000074
:102DE000D65E0000F85E00001A5F00003B5F000046
:102DF0005D5F00007E5F0000A05F0000C15F00001B
:102E0000E25F0000046000002560000046600000F2
:102E10006760000088600000A9600000CA600000D0
:102E2000EB6000000C6100002D6100004D610000AE
:102E30006E6100008E610000AF610000CF61000094
:102E4000F06100001062000030620000516200007A
:102E50007162000091620000B1620000D162000066
:102E6000F162000011630000306300005063000055
:102E7000706300008F630000AF630000CE6300004A
:102E8000EE6300000D6400002D6400004C6400003F
:102E90006B6400008A640000A9640000C86400003C
:102EA000E764000006650000256500004465000039
:102EB0006265000081650000A0650000BE6500003D
:102EC000DD650000FB650000196600003866000043
:102ED000566600007466000092660000B06600004E
:102EE000CE660000EC6600000A670000286700005C
:102EF0004567000063670000816700009E6700006F
:102F0000BC670000D9670000F76700001468000084
:102F1000316800004E6800006B680000886800009F
:102F2000A5680000C2680000DF680000FC680000BF
:102F30001969000035690000526900006E690000DF
:102F40008B690000A7690000C4690000E069000007
:102F5000FC690000186A0000346A0000506A000032
:102F60006C6A0000886A0000A46A0000C06A000061
:102F7000DB6A0000F76A0000136B00002E6B000094
:102F80004A6B0000656B0000806B00009C6B0000CA
:102F9000B76B0000D26B0000ED6B0000086C000006
:102FA000236C00003E6C0000586C0000736C000045
:102FB0008E6C0000A86C0000C36C0000DD6C00008B
:102FC000F86C0000126D00002C6D0000476D0000D1
:102FD000616D00007B6D0000956D0000AF6D00001D
:102FE000C96D0000E36D0000FC6D0000166E00006E
:102FF000306E0000496E0000636E00007C6E0000C1
:10300000956E0000AF6E0000C86E0000E16E00001B
:10301000FA6E0000136F00002C6F0000456F000077
:103020005E6F0000766F00008F6F0000A86F0000D9
:10303000C06F0000D96F0000F16F00000970000040
:10304000227000003A700000527000006A700000A8
:10305000827000009A700000B2700000CA70000018
:10306000E1700000F970000011710000287100008B
:1030700040710000577100006E7100008671000001
:103080009D710000B4710000CB710000E27100007E
:10309000F971000010720000267200003D720000FD
:1030A000547200006A720000817200009772000082
:1030B000AE720000C4720000DA720000F07200000C
:1030C000067300001C730000327300004873000098
:1030D0005E73000074730000897300009F7300002A
:1030E000B5730000CA730000DF730000F5730000C1
:1030F0000A7400001F74000034740000497400005A
:103100005E74000073740000887400009D740000F9
:10311000B1740000C6740000DB740000EF7400009E
:1031200003750000187500002C7500004075000044
:1031300054750000687500007C75000090750000F3
:10314000A4750000B8750000CC750000DF750000A4
:10315000F3750000067600001A7600002D76000058
:103160004076000053760000677600007A76000013
:103170008D760000A0760000B2760000C5760000D3
:10318000D8760000EA760000FD7600001077000097
:10319000227700003477000047770000597700005D
:1031A0006B7700007D7700008F770000A17700002B
:1031B000B3770000C4770000D6770000E8770000FE
:1031C000F97700000B7800001C7800002E780000D2
:1031D0003F780000507800006178000072780000AD
:1031E0008378000094780000A5780000B67800008D
:1031F000C6780000D7780000E7780000F878000073
:103200000879000019790000297900003979000057
:103210004979000059790000697900007979000046
:103220008979000098790000A8790000B879000039
:10323000C7790000D7790000E6790000F579000031
:10324000047A0000147A0000237A0000327A000029
:10325000417A00004F7A00005E7A00006D7A00002B
:103260007C7A00008A7A0000997A0000A77A000030
:10327000B57A0000C47A0000D27A0000E07A00003B
:10328000EE7A0000FC7A00000A7B0000187B000048
:10329000257B0000337B0000417B00004E7B00005B
:1032A0005C7B0000697B0000767B0000837B000074
:1032B000917B00009E7B0000AB7B0000B87B000090
:1032C000C47B0000D17B0000DE7B0000EB7B0000B4
:1032D000F77B0000047C0000107C00001C7C0000D8
:1032E000297C0000357C0000417C00004D7C000002
:1032F000597C0000657C0000707C00007C7C000034
:10330000887C0000937C00009F7C0000AA7C000069
:10331000B67C0000C17C0000CC7C0000D77C0000A3
:10332000E27C0000ED7C0000F87C0000037D0000E2
:103330000E7D0000187D0000237D00002E7D000022
:10334000387D0000427D00004D7D0000577D00006B
:10335000617D00006B7D0000757D00007F7D0000B9
:10336000897D0000937D00009C7D0000A67D00000B
:10337000B07D0000B97D0000C27D0000CC7D000062
:10338000D57D0000DE7D0000E77D0000F07D0000BF
:10339000F97D0000027E00000B7E0000137E00001D
:1033A0001C7E0000257E00002D7E0000367E000081
:1033B0003E7E0000467E00004E7E0000567E0000ED
:1033C0005E7E0000667E00006E7E0000767E00005D
:1033D0007E7E0000857E00008D7E0000947E0000D1
:1033E0009C7E0000A37E0000AA7E0000B27E00004A
:1033F000B97E0000C07E0000C77E0000CE7E0000C7
:10340000D47E0000DB7E0000E27E0000E87E00004B
:10341000EF7E0000F57E0000FC7E0000027F0000D1
:10342000087F00000E7F0000147F00001A7F00005C
:10343000207F0000267F00002C7F0000317F0000ED
:10344000377F00003C7F0000427F0000477F000084
:103450004C7F0000527F0000577F00005C7F00001F
:10346000617F0000667F00006A7F00006F7F0000C0
:10347000747F0000787F00007D7F0000817F000066
:10348000867F00008A7F00008E7F0000927F000010
:10349000967F00009A7F00009E7F0000A27F0000C0
:1034A000A67F0000A97F0000AD7F0000B07F000074
:1034B000B47F0000B77F0000BB7F0000BE7F00002C
:1034C000C17F0000C47F0000C77F0000CA7F0000EA
:1034D000CD7F0000CF7F0000D27F0000D57F0000AD
:1034E000D77F0000D97F0000DC7F0000DE7F000076
:1034F000E07F0000E27F0000E47F0000E67F000044
:10350000E87F0000EA7F0000EC7F0000EE7F000013
:10351000EF7F0000F17F0000F27F0000F37F0000EA
:10352000F57F0000F67F0000F77F0000F87F0000C5
:10353000F97F0000FA7F0000FB7F0000FB7F0000A6
:10354000FC7F0000FD7F0000FD7F0000FE7F00008B
:10355000FE7F0000FE7F0000FE7F0000FE7F000077
:10356000FF7F000000000000EFFF000004000000EB
:1035700002000000E5FF0000E1FF0000FCFF00008A
:10358000FAFF0000D4FF0000CFFF0000F7FF0000AB
:10359000F8FF0000C3FF0000C0FF000000000000B3
:1035A00006000000BFFF0000C1FF00002500000072
:1035B00035000000D4FF0000DDFF000071000000B6
:1035C0008A000000000000000C000000D80000008D
:1035D000F30000002C000000310000003701000063
:1035E0004901000027000000160000005B010000F8
:1035F00057010000B8FF000085FF0000190100001E
:10360000F8000000B9FE000062FE00006C0000003F
:103610003700000038FD0000C8FC000093FF0000E8
:1036200066FF000078FB00000AFB00001CFF0000A2
:1036300029FF0000EEF90000A2F9000000000000E0
:10364000A200000016F9000005F900007304000054
:10365000E706000043F9000079F90000A41C00000F
:10366000FF3F00006F310000F7FA000094D800001F
:10367000D0E4000091FC000024FD00004EF20000A8
:103680009BF40000E7FE000075FF000061F90000F8
:103690008FFA0000F50000005E01000043FD00000D
:1036A000F2FD00004E020000800200006AFF0000F0
:1036B000BFFF0000C7020000C40200004E0000006F
:1036C0006300000080020000580200005B00000060
:1036D0004B000000C7010000920100000000000044
:1036E000E6FF0000F9000000CA0000009BFF000098
:1036F00088FF0000580000003A00000063FF00004F
:103700005FFF000000000000F5FF000064FF000004
:103710006CFF0000E9FF0000EAFF00008CFF0000E2
:1037200099FF0000F6FF0000FAFF0000BEFF000056
:10373000C9FF0000090000000D000000E4FF0000C8
:10374000ECFF00001600000017000000FAFF000068
:10375000FEFF00001A0000001A0000000200000036
:103760000000000000000000FCFF0000FDFF000062
:10377000E5FF0000E6FF0000020000000500000079
:10378000E8FF0000EAFF0000140000001B0000003A
:10379000F3FF0000F6FF00003600000042000000CA
:1037A000050000000A00000067000000740000002F
:1037B0001600000016000000930000009B000000AF
:1037C0000A000000FFFF0000A00000009C000000B5
:1037D000C5FF0000A8FF00007700000065000000A2
:1037E00036FF000007FF00001A0000000000000084
:1037F0006EFE000038FE0000B5FF0000A4FF0000D0
:10380000A8FD000080FD00009DFF0000B1FF00004A
:103810003CFD000038FD0000410000009600000063
:1038200080FD0000B2FD00000E020000BD0200009D
:10383000A2FE00000AFF0000700500009E060000C6
:103840008A00000018010000650B0000B10D0000A7
:10385000DC0200006E0300002F1B00006B2700003D
:103860000905000091CE000001C000005BE30000EC
:1038700086060000BC06000018F900008CFB000062
:10388000FB060000EA0600005DFF000000000000EB
:103890005E06000011060000D6000000E3000000F4
:1038A000F504000087040000990000006C0000008F
:1038B00037030000C8020000C9FF000094FF0000A9
:1038C0009D0100004601000008FF0000E7FE000027
:1038D0007B00000048000000A9FE0000A4FE0000DC
:1038E000EAFF0000D9FF0000B7FE0000C8FE00009C
:1038F000CEFF0000D3FF00000CFF000028FF0000F7
:10390000F3FF0000FFFF000076FF00008FFF0000C4
:10391000230000002C000000CAFF0000DAFF0000B6
:103920003F00000041000000F9FF0000000000001F
:10393000400000003D0000000800000008000000FA
:10394000300000002B000000050000000400000013
:103950001E0000001A000000FEFF0000FCFF000037
:103960000000000000000000000000000000000057
:103970000000000000000000000000000000000047
:103980000000000000000000000000000000000037
:103990000000000000000000000000000000000027
:1039A0000000000000000000000000000000000017
:1039B0000000000000000000000000000000000007
:1039C0000000000000000000FFFF000001000000F8
:1039D000000000000000000000000000FFFF0000E9
:1039E0000100000000000000FFFF000000000000D8
:1039F000FFFF00000200000000000000FEFF0000CA
:103A000000000000FFFF000002000000FFFF0000B8
:103A1000FFFF000000000000FFFF000002000000A8
:103A2000FDFF00000000000000000000000000009A
:103A300002000000FBFF000000000000000000008A
:103A40000000000001000000FBFF0000FDFF00007F
:103A5000000000000100000000000000FCFF00006A
:103A6000F9FF00000000000001000000FFFF00005F
:103A7000FEFF0000F9FF0000000000000100000050
:103A8000FFFF000000000000FEFF0000000000003B
:103A90000000000000000000000000000000000026
:103AA00000000000FFFF000002000000FDFF00001A
:103AB000FAFF000000000000FEFF0000050000000B
:103AC000F8FF0000F1FF000000000000FEFF000012
:103AD00007000000F1FF0000F1FF000000000000FF
:103AE000FEFF000009000000EDFF0000FEFF0000E7
:103AF000000000000100000008000000EEFF0000D0
:103B000008000000000000000500000004000000A4
:103B1000F6FF000000000000000000000B000000A5
:103B2000FBFF000004000000EFFF000000000000A9
:103B300012000000EEFF000012000000EEFF000087
:103B4000000000001A000000DFFF00001B00000062
:103B5000070000000000000020000000CFFF000070
:103B60001B000000230000000000000024000000F3
:103B7000C4FF0000100000001F0000000000000053
:103B800022000000BFFF0000000000000000000055
:103B90000000000019000000C3FF0000F6FF000055
:103BA000F6FF00000000000009000000D3FF000045
:103BB000FCFF00001E00000000000000F0FF0000FD
:103BC000EBFF0000150000005500000000000000A1
:103BD000D2FF00000A0000003E0000005B00000071
:103BE00000000000B0FF0000290000006900000094
:103BF000260000000000000090FF000042000000CE
:103C000084000000000000000000000077FF0000BA
:103C100050000000810000002D00000000000000A6
:103C20006AFF0000510000005D00000088000000F5
:103C30000000000070FF00004300000027000000AB
:103C40009E000000000000008AFF00002B00000022
:103C5000F6FF00004500000000000000BBFF000070
:103C600012000000E4FF0000E4FF0000000000007C
:103C70000000000000000000FFFF0000FFFF000048
:103C8000000000005400000001000000410000009E
:103C90008100000000000000AC0000001A000000DD
:103CA0008B000000B700000000000000FF000000D3
:103CB0004D000000B30000003100000000000000D3
:103CC0004101000094000000940000006BFF000020
:103CD0000000000064010000E10000002600000078
:103CE0004FFF000000000000610100002001000003
:103CF00080FF0000FFFF0000000000003301000013
:103D00003C010000DAFE00007B0000000000000023
:103D1000D90000002101000074FE0000D3FF000064
:103D20000000000059000000C30000007AFE0000FF
:103D30007AFE000000000000C1FF00001F0000002C
:103D4000E9FE0000F3FD0000000000001FFF00007E
:103D500042FF00008BFF0000E4FE000000000000B6
:103D600089FE000048FE0000000000000000000086
:103D70000000000010FE000054FD0000E9FF0000FC
:103D80006BFF000000000000C7FD000091FC000078
:103D900015FF00003FFD000000000000BAFD00001C
:103DA00029FC00009EFD0000E2FB00000000000076
:103DB000EEFD000039FC0000F6FB00003CFD0000B9
:103DC0000000000062FE0000D0FC0000C5FA000008
:103DD000DBFF0000000000000AFF0000E5FD00001E
:103DE000B4FA00000100000000000000D5FF000050
:103DF0005EFF00002AFC00002BFC00000000000019
:103E0000AC0000000B01000018FF000013F80000D8
:103E10000000000076010000B2020000F102000084
:103E2000E4F90000000000001B020000160400007E
:103E3000CB060000A703000000000000870200007E
:103E400004050000A1090000D20F000000000000DE
:103E5000AC02000057050000AC0A00005715000036
:103E6000000000008702000004050000A109000016
:103E7000D20F0000000000001B020000160400002A
:103E8000CB060000A7030000000000007601000040
:103E9000B2020000F1020000E4F90000000000009E
:103EA000AC0000000B01000018FF000013F8000038
:103EB00000000000D5FF00005EFF00002AFC0000AB
:103EC0002BFC0000000000000AFF0000E5FD0000E0
:103ED000B4FA0000010000000000000062FE0000D3
:103EE000D0FC0000C5FA0000DBFF0000000000006D
:103EF000EEFD000039FC0000F6FB00003CFD000078
:103F000000000000BAFD000029FC00009EFD00003A
:103F1000E2FB000000000000C7FD000091FC000073
:103F200015FF00003FFD00000000000010FE000033
:103F300054FD0000E9FF00006BFF000000000000DE
:103F400089FE000048FE00000000000000000000A4
:103F5000000000001FFF000042FF00008BFF000078
:103F6000E4FE000000000000C1FF00001F00000090
:103F7000E9FE0000F3FD0000000000005900000011
:103F8000C30000007AFE00007AFE0000000000007E
:103F9000D90000002101000074FE0000D3FF0000E2
:103FA00000000000330100003C010000DAFE0000C8
:103FB0007B00000000000000610100002001000003
:103FC00080FF0000FFFF000000000000640100000F
:103FD000E1000000260000004FFF0000000000008C
:103FE0004101000094000000940000006BFF0000FD
:103FF00000000000FF0000004D000000B3000000C2
:104000003100000000000000AC0000001A000000B9
:104010008B000000B700000000000000540000000A
:1040200001000000410000008100000000000000CD
:104030000000000000000000FFFF0000FFFF000084
:1040400000000000BBFF000012000000E4FF0000C1
:10405000E4FF0000000000008AFF00002B000000C9
:10406000F6FF0000450000000000000070FF0000A7
:1040700043000000270000009E0000000000000038
:104080006AFF0000510000005D0000008800000091
:104090000000000077FF00005000000081000000D9
:1040A0002D0000000000000090FF00004200000012
:1040B000840000000000000000000000B0FF0000CD
:1040C0002900000069000000260000000000000038
:1040D000D2FF00000A0000003E0000005B0000006C
:1040E00000000000F0FF0000EBFF000015000000E2
:1040F000550000000000000009000000D3FF000090
:10410000FCFF00001E00000000000000190000007D
:10411000C3FF0000F6FF0000F6FF000000000000F3
:1041200022000000BFFF00000000000000000000AF
:104130000000000024000000C4FF00001000000088
:104140001F0000000000000020000000CFFF000062
:104150001B00000023000000000000001A00000007
:10416000DFFF00001B00000007000000000000004F
:1041700012000000EEFF000012000000EEFF000041
:10418000000000000B000000FBFF00000400000026
:10419000EFFF000000000000050000000400000028
:1041A000F6FF000000000000000000000100000019
:1041B00008000000EEFF0000080000000000000002
:1041C000FEFF000009000000EDFF0000FEFF000000
:1041D00000000000FEFF000007000000F1FF0000EB
:1041E000F1FF000000000000FEFF000005000000DD
:1041F000F8FF0000F1FF000000000000FFFF0000DA
:1042000002000000FDFF0000FAFF000000000000B7
:10421000000000000000000000000000000000009E
:104220000000000001000000FFFF0000000000008F
:10423000FEFF00000000000001000000FFFF000082
:10424000FEFF0000F9FF0000000000000100000078
:1042500000000000FCFF0000F9FF0000000000006B
:104260000000000001000000FBFF0000FDFF000057
:10427000000000000000000002000000FBFF000042
:104280000000000000000000FFFF0000020000002E
:10429000FDFF00000000000000000000FFFF000024
:1042A00002000000FFFF0000FFFF00000000000010
:1042B000FFFF00000200000000000000FEFF000001
:1042C00000000000FFFF00000100000000000000EF
:1042D000FFFF000000000000FFFF000001000000E1
:1042E00000000000000000000000000000000000CE
:1042F00000000000000000000000000000000000BE
:1043000000000000000000000000000000000000AD
:10431000000000000000000000000000000000009D
:10432000000000000000000000000000000000008D
:10433000000000000000000000000000000000007D
:10434000000000000000000000000000000000006D
:10435000010200000408000010200000408000005E
:1043600000800000C0E00000F0F80000FCFE00004B
:10437000000000000000000000000000005F0000DE
:10438000000000000007000000070000001400000B
:104390007F1400007F140000242A00007F2A000000
:1043A0001223000013080000646200003649000078
:1043B000552200005000000005030000000000002E
:1043C000001C00002241000000000000412200000B
:1043D0001C000000082A00001C2A00000808000039
:1043E000083E0000080800000050000030000000F7
:1043F0000008000008080000080800000060000035
:10440000600000000020000010080000040200000E
:104410003E510000494500003E000000427F000080
:1044200040000000426100005149000046210000A8
:10443000414500004B31000018140000127F0000BD
:104440001027000045450000453900003C4A0000A7
:104450004949000030010000710900000503000017
:10446000364900004949000036060000494900006D
:10447000291E000000360000360000000000000089
:104480005636000000000000000800001422000062
:104490004114000014140000141400004122000014
:1044A000140800000002000001510000090600008D
:1044B00032490000794100003E7E000011110000E9
:1044C000117E00007F49000049490000363E00008F
:1044D00041410000412200007F41000041220000D4
:1044E0001C7F000049490000494100007F0900008D
:1044F00009010000013E000041410000513200006E
:104500007F080000080800007F000000417F0000D5
:104510004100000020400000413F0000017F0000FA
:1045200008140000224100007F40000040400000CD
:10453000407F000002040000027F00007F040000B2
:10454000081000007F3E000041410000413E000095
:104550007F09000009090000063E000041510000EB
:10456000215E00007F090000192900004646000076
:104570004949000049310000010100007F010000AD
:10458000013F000040400000403F00001F200000AD
:10459000402000001F7F000020180000207F000046
:1045A0006314000008140000630300000478000096
:1045B0000403000061510000494500004300000071
:1045C000007F0000414100000204000008100000CC
:1045D00020410000417F00000000000004020000B4
:1045E0000102000004400000404000004040000084
:1045F00000010000020400000020000054540000EC
:10460000547800007F48000044440000383800001F
:1046100044440000442000003844000044480000A6
:104620007F3800005454000054180000087E000039
:10463000090100000208000014540000543C00006E
:104640007F0800000404000078000000447D0000A2
:104650004000000020400000443D00000000000039
:104660007F10000028440000004100007F4000004F
:10467000007C000004180000047800007C080000A2
:10468000040400007838000044440000443800006E
:104690007C1400001414000008080000141400002A
:1046A000187C00007C08000004040000084800009A
:1046B0005454000054200000043F00004440000017
:1046C000203C000040400000207C00001C20000036
:1046D000402000001C3C000040300000403C000036
:1046E0004428000010280000440C00005050000036
:1046F000503C000044640000544C000044000000A2
:104700000836000041000000000000007F000000AB
:10471000000000004136000008000000080800000A
:104720002A1C0000080800001C2A000008080000DD
:104730002F0F00002000000000F80000F8880000A3
:10474000A0F80000E00000000000000000000000F1
:104750000000000000000000000000000000000059
:104760000000000000000000000000000000000049
:104770000000000000000000000000000000000039
:104780000000000000000000000000000000000029
:104790000000000000000000000000000000000019
:1047A000000000000000000000000000000F0000FA
:1047B0002F00000020A8000000A80000A8F80000BA
:1047C000A8000000F8000000000000000000000049
:1047D00000000000000000000000000000000000D9
:1047E00000000000000000000000000000000000C9
:1047F00000000000000000000000000000000000B9
:1048000000000000000000000000000000000000A8
:104810000000000000000000000000000000000098
:104820000000000000F8000000A000000FEF0000F2
:10483000525300004C200000644200006D3A00001A
:104840000025000073200000252D000034690000C1
:1048500000560000322E0000300000002020000032
:104860002020000020200000202000002020000048
:104870002020000020200000202000002020000038
:1048800020000000536500007475000070200000D7
:104890002020000020200000202000002020000018
:1048A00020200000202000002000000045780000AB
:1048B000697400002020000020200000202000005B
:1048C00020200000202000002020000020200000E8
:1048D00020000000536100007665000020430000C6
:1048E000686100006E670000657300002020000012
:1048F000202000002020000020000000525800006E
:10490000204100006D70000020540000726900001A
:104910006D2000002020000020200000202000004A
:104920002000000052580000205000006861000084
:104930007365000020540000726900006D200000C3
:10494000202000002020000020000000545800001B
:10495000204100006D7000002054000072690000CA
:104960006D200000202000002020000020200000FA
:104970002000000054580000205000006861000032
:104980007365000020540000726900006D20000073
:1049900020200000202000002000000054580000CB
:1049A000204D00006963000020470000616900009D
:1049B0006E200000202000002020000020200000A9
:1049C0002000000054580000204300005720000041
:1049D00047610000696E00002020000020200000D8
:1049E0002020000020200000200000004C69000072
:1049F0006E6500002D4900006E2000004761000038
:104A0000696E00002020000020200000202000000F
:104A10002000000050470000413000002047000007
:104A2000616900006E2000002020000020200000AE
:104A30002020000020200000200000004669000027
:104A40006C7400002042000057200000202000006D
:104A50002020000020200000202000002020000056
:104A60002000000042610000636B00006C690000E0
:104A70006768000074200000202000002020000053
:104A800020200000202000002000000052650000CF
:104A9000737400006F720000652000004465000020
:104AA00066610000756C0000747300002020000037
:104AB0002000000025360000640000005047000080
:104AC00041470000616900006E300000203D000099
:104AD000202500003264000000460000696C0000E0
:104AE00074650000722000004E7500006D3A0000F1
:104AF000202500003264000000200000202000007B
:104B000032350000304800007A000000202000000C
:104B10002035000030300000487A000000200000FE
:104B2000202000003130000030300000487A0000C2
:104B30000020000020200000323000003030000053
:104B4000487A000000420000616300006B6C0000C6
:104B50006967000068740000204C00006576000062
:104B6000656C00003A20000025320000640000005F
:104B7000FF7F000000000000D97F0000B8F90000AE
:104B8000627F000074F300009D7E000038ED00009D
:104B90008A7D000007E700002A7C0000E6E00000B4
:104BA0007D7A0000D8DA000085780000E1D40000AA
:104BB0004276000004CF0000B673000046C9000032
:104BC000E3700000A9C30000CA6D000032BE0000FF
:104BD0006E6A0000E3B80000D0660000C0B30000B9
:104BE000F2620000CCAE0000D75E00000AAA00000E
:104BF000825A00007EA50000F655000029A10000A1
:104C0000345100000E9D0000404C0000309900001F
:104C10001D47000092950000CE4100003692000032
:104C2000573C00001D8F0000BA3600004A8C00007F
:104C3000FC300000BE8900001F2B00007B870000B5
:104C400028250000838500001A1F0000D68300007D
:104C5000F918000076820000C8120000638100008D
:104C60008C0C00009E800000480600002780000099
:104C70000000000000800000B8F90000278000005C
:104C800074F300009E80000038ED00006381000096
:104C900007E7000076820000E6E00000D68300000F
:104CA000D8DA000083850000E1D400007C87000092
:104CB00004CF0000BE89000046C900004A8C0000F5
:104CC000A9C300001D8F000032BE00003692000014
:104CD000E3B8000092950000C0B3000031990000D5
:104CE000CCAE00000E9D00000AAA000029A1000021
:104CF0007EA500007EA5000029A100000AAA0000F0
:104D00000E9D0000CCAE000031990000C0B3000041
:104D100092950000E3B800003692000032BE000019
:104D20001D8F0000A9C300004A8C000046C9000086
:104D3000BE89000004CF00007C870000E1D40000A1
:104D400083850000D8DA0000D6830000E6E000008A
:104D50007682000007E700006381000038ED000064
:104D60009E80000074F3000027800000B8F9000066
:104D7000435700002D4C000000430000572D000059
:104D800055000000202000002D570000494400007D
:104D900045000000202000002D4E00004152000080
:104DA00000530000534200002D4C0000005300004F
:104DB000534200002D550000004400004947000008
:104DC0002D4C000000440000494700002D55000014
:104DD000000000002C2D00002E30000031320000B9
:104DE0003435000036380000393A00003C3D000000
:104DF0003E24000025260000282900002A2C00005F
:104E00002D2E000030310000323400003536000015
:104E10007FAC0000238000005F1000007FAC00002A
:104E2000237F0000A0F0000080A70000B800000071
:104E3000404100004244000045460000484900004F
:104E40004A4C00004D4E0000505100005238000006
:104E5000393A00003C3D00003E4000004142000065
:104E60004445000046480000494A00007FAA00006F
:104E70006E80000065B200007FAA00006E7F000017
:104E80009A4E000080AB0000220000005455000044
:104E900056580000595A00005C5D00005E6000003A
:104EA0006162000064650000664C00004D4E000029
:104EB000505100005254000055560000585900004F
:104EC0005A5C00005D5E00007FAA00006E8000005A
:104ED000825C00007FAA00006E7F00007DA40000BD
:104EE00080AB000022000000686900006A6C0000CE
:104EF0006D6E000070710000727400007576000025
:104F0000787900007A60000061620000646500004A
:104F100066680000696A00006C6D00006E70000039
:104F2000717200007FAA00006E800000960F0000E2
:104F30007FAA00006E7F000069F1000080AB0000D6
:104F4000220000007C7D00007E080000090A0000AD
:104F50000C0D00000E1000001112000014150000CE
:104F60001674000075760000787900007A7C0000E5
:104F70007D7E0000080900000A0C00000D0E0000F4
:104F80007FAA00006E800000E69D00007FAA00005E
:104F90006E7F00001963000080AB0000220000005B
:104FA00000000000003F00000AD70000233C000082
:104FB00000000000003F00000AD70000233C000072
:104FC0006F120000833B00006F120000833B000063
:104FD000000000004843000059B10000AE38000056
:104FE0000AD70000233C0000CD000000238700000A
:104FF000883C0000C7BB00007B3F000000FC0000B5
:10500000FF460000CDCC0000CC3E0000187200002E
:10501000313F0000EBA80000AA3D00000E00FA009E
:10502000881F7800D2C2BF000080FB004400DE0071
:10503000614060000080FB0010079800D2C2BF00F2
:105040000080FB004300DE00614060000080FB0048
:10505000000F78001E00E0000300320040C0B300E3
:10506000E3020700020037004ADABF00E00207004F
:105070001EBBA8001E9BA9000040EB0070479800D3
:1050800076003700FE40900080CBB30000C0700077
:105090009A02070000C4B300980207007E40900007
:1050A000E44F50000D0036000040EB00104F980018
:1050B000050037000040EB009F0207001E489000EB
:1050C0000040E800104F98009E489000F0C3B300E5
:1050D00080CF5000F7FF36005D0037007E40900023
:1050E000E44F500026003A000040EB00104F9800BB
:1050F0001E00370041B12100914078001E48900009
:10510000814F50001000360061B1210091407800BD
:105110001E489000814F50000B0031001E0090008F
:105120000000E00008003A001E4890000080FB00EC
:105130008000400080392A00614078000014A000FF
:105140007D020700060037001E4890000080FB002B
:105150008000400080392A00614078007602070014
:105160001E4890000040E800104F98009E489000B4
:10517000F0C3B30080CF5000DEFF360034003700AC
:105180000040EB00104F98002D0037001E489000A3
:105190000080FB0080004000C092210000804000A1
:1051A00010007800004F98000E4890000080FB002F
:1051B0004300DE0060479800EE40900030C0B3002E
:1051C00001405000504798008E4890006E4090007B
:1051D0000080FB004300DD0000C050004047980005
:1051E000FE4090005E40900080CF500002003100F1
:1051F0000040EB0050020700FE4090005E4090002F
:1052000080CF500005003A004E4090008080FB00A7
:10521000001B2A006140780047020700FE40900012
:105220005E40900080CF50000200360000C0EB00CE
:10523000410207001E4890000040E800104F98000F
:105240009E489000F0C3B30080CF5000CFFF3600DF
:105250007E4090000040E800704798007E4090003B
:10526000E74F500087FF36001EBBA9001E9BA80019
:105270000040EB007047980079003700FE40900036
:1052800080CBB30000C070001C02070000C4B30054
:105290001A0207007E409000E44F50000D003600D7
:1052A0000040EB00104F9800050037000040EB0075
:1052B000210207001E4890000040E800104F9800AF
:1052C0009E489000F0C3B30080CF5000F7FF360037
:1052D000600037007E409000E44F500028003A0004
:1052E0000040EB00104F98002000370051B1210022
:1052F000914078001E489000814F50001100360008
:1053000071B12100914078001E489000814F5000FB
:105310000C0031001E0090000000E0000900320087
:105320001E4890000080FB00000040008000E80064
:1053300080392A00614078000014A000FE010700B7
:10534000070037001E4890000080FB00000040006E
:105350008000E80080392A0061407800F6010700EB
:105360001E4890000040E800104F98009E489000B2
:10537000F0C3B30080CF5000DCFF360035003700AB
:105380000040EB00104F98002E0037001E489000A0
:105390000080FB000004B00080004000C0922100AB
:1053A0000080400010007800004F98000E489000E8
:1053B0000080FB004300DE0060479800EE40900054
:1053C00030C0B30001405000504798008E48900014
:1053D0006E4090000080FB004300DD0000C05000E4
:1053E00040479800FE4090005E40900080CF500003
:1053F000020031000040EB00CF010700FE409000AA
:105400005E40900080CF500005003A004E40900072
:105410008080FB00001B2A0061407800C601070065
:10542000FE4090005E40900080CF500002003600A9
:1054300000C0EB00C00107001E4890000040E800DB
:10544000104F98009E489000F0C3B30080CF5000EA
:10545000CEFF36007E4090000040E8007047980084
:105460007E409000E74F500084FF36003DDBBF00D8
:10547000664060000004E00046003A0041D580002C
:10548000B0032000808F50001900340038B980002C
:105490006140B9005BED0700500798006107980074
:1054A0000800E00007003D0002002000037824000F
:1054B0005E009000EE0090007EED0700500798001F
:1054C000610798005E009000EE00900032332300E8
:1054D00033052C00D4ED070002002000032F240028
:1054E00074ED0700C0D88800D1D888000B003700C1
:1054F00040D58000CF80DE0042ED07000200200092
:1055000003F02300C8ED070002002000032224005E
:1055100068ED0700C0D88800D1D88800C0D88000C6
:10552000D1D88000F4ED0700E0D88800E0D88000F2
:105530000000EA00801F780080412A00801F780068
:1055400010422A00801F780000A92100A2F0070065
:10555000E68757008041EB0062C0B3008040EB005B
:1055600000A92100210107008041EB0072C0B300B7
:105570008040EB00C0A721001C0107008041EB0028
:1055800072C0B300F1C0B30090422A0017010700B7
:1055900013003700C0A72100E1422A0013000900D0
:1055A000315878008041EB0062C0B3008040EB00CE
:1055B00040A521000D0107008041EB0072C0B3003F
:1055C0008040EB0080A62100080107008041EB002D
:1055D00052C0B3008040EB00C0A7210003010700C8
:1055E0004F0478000080FA00000006000600FA0070
:1055F000000F7800214798003247980043479800F1
:105600005447980023003700BE4090003E40900071
:105610000040E900304798001E007800A2002000FA
:10562000811F7800110009000200D80000017800F5
:1056300001007800CF0078000043B000DE41900008
:105640004E419000960007001E007800A200200046
:10565000110009000200D800000F78002E409000D1
:105660000040E900204798002E4090000004E00030
:1056700008003A00BE4090003E4090000040E90023
:1056800030479800DE4190004E419000E0C2B300E8
:10569000830007001E00E000DBFF3C002E4090006E
:1056A0000004E000D8FF3D000080FA000000060082
:1056B0000200FA001EBBA8001E9BA9000040EB00E0
:1056C000004F78001200370080CBB3001E407000FE
:1056D0000A01070000C4B300080107000040EB0006
:1056E00010479800050037000040EB00120107004A
:1056F0001E4090000040E800104798009E40900037
:10570000F0C3B30080CF5000F7FF36001E4FE80013
:1057100070C0B3009E4F1000EBFF36001EBBA90007
:105720001E9BA8000040EB00004F780012003700DD
:1057300080CBB3001E407000F000070000C4B3002F
:10574000EE0007000040EB0010479800050037000E
:105750000040EB00F80007001E4090000040E80009
:10576000104798009E409000F0C3B30080CF5000D7
:10577000F7FF36001E4FE80070C0B3009E4F1000C8
:10578000EBFF36000080FA00000006000400FA007B
:105790001EBBA8001E9BA9000040EB00104798000C
:1057A000190037009E40900080CBB30000C070000D
:1057B000D200070000C4B300D00007000040EB0097
:1057C0002047980009003700AE40900000C4B300A5
:1057D00000C07000C90007001EC0EA00D600070024
:1057E0002E4090000040E80020479800AE40900016
:1057F000F0C3B30080CF5000F3FF36001E4090008E
:105800000040E800104798001E409000E74F50000D
:10581000E4FF36001EBBA9001E9BA8000040EB0061
:1058200010479800190037009E40900080CBB300CD
:1058300000C07000B100070000C4B300AF00070053
:105840000040EB002047980009003700AE40900070
:1058500000C4B30000C07000A80007001EC0EA002A
:10586000B50007002E4090000040E8002047980057
:10587000AE409000F0C3B30080CF5000F3FF36007D
:105880001E4090000040E800104798001E40900025
:10589000E74F5000E4FF36000080FA0000000600E9
:1058A0000600FA00204798003147980042479800C8
:1058B000534798003E409000F34F500002003600DE
:1058C0000040EB00304798004E4090006740600079
:1058D000404798003E409000E94F50000A003E00CB
:1058E0001EBBA8001E9BA9003E4090000080FB004C
:1058F0006600B900E440400000C4B30000C070007E
:105900007E0007000B0037001EBBA9001E9BA800ED
:105910003E4090000080FB006600B90080407800A7
:1059200040CCB30080C0400000C4B30000C0700091
:1059300072000700CE40900080CBB30000C0700022
:105940006E0007000040EB00004F78001A0037009F
:105950005E4090000004E0000B003A002E409000F2
:105960008080FB0000FE2F00008040001E81FB00B5
:105970006500B90082004000801B2A006140780069
:105980006D0007000B0037002E4090008080FB0068
:1059900000FE2F00008040001E81FB006500B90062
:1059A00082004000801B2A006140780000C0EA00AD
:1059B000610007001E4FE80040C0B3009E4F10007A
:1059C000E3FF36005E4090000004E00003003A0070
:1059D0000040EB00580007000200370000C0EB0059
:1059E000550007000080FA00000006000800FA00D9
:1059F0001007980041479800524798006347980065
:105A000008003700CE4090004E4090000040E80073
:105A1000404798001E407800EE4190005E419000A3
:105A20009FFF07001E009000104F78001E40780076
:105A3000704798007E4090000004E00002003200B1
:105A400010C0B300704798007E4090009E00900008
:105A50008100E800110798000004E000E9FF3A0027
:105A60000080FA00000006000400FA0000C2B30043
:105A7000204798000EFF07000040EB00004F780021
:105A8000190037000040EB00104798001200370063
:105A90002E4290002E4090000040E80020479800E1
:105AA0008041EB001E4178009E4090000440780049
:105AB0007BFF0700AE40900000C8B30080CF5000CD
:105AC00002003A0000C2B300204798001E40900038
:105AD0000040E800104798001E409000F34F50002F
:105AE000EBFF36001E4FE80070C0B3009E4F100061
:105AF000E4FF36000080FA00000006000200FA0011
:105B0000004F78001E3BA9001E5BA9001E7BA80069
:105B1000E1B121009140780020C1B30016100700C8
:105B20009E40780030C1B300131007001100070039
:105B30000080FA00000006000200FA00004F780022
:105B40001E3BA8001E5BA9001E7BA800E1B121003E
:105B50009140780020C1B300071007009E407800F4
:105B600030C1B30004100700020007000080FA00F3
:105B7000000006000000FA001E1BA8001E7BA80003
:105B8000E1B121009140780020C1B300FA0F070075
:105B90001E1BA9001E7BA800E1B1210091407800E6
:105BA00020C1B300F40F07000080FA0000000600D7
:105BB0000000FA00070B07001EBBA8001E9BA900EF
:105BC000F0C3B300CDFF070000CCB300CBFF07004C
:105BD0001EBBA9001E9BA800F0C3B300C7FF0700AF
:105BE00000CCB300C5FF07000080FA0000000600EB
:105BF0000400FA00004F78001E80FB001007980098
:105C00001E009000E10F5000170032001E009000AF
:105C1000E10F500004003C001E0090000000E00076
:105C2000080032002B0037001E009000E20F5000E9
:105C3000160032001E009000E30F50001C003200DE
:105C40002400370070C3B30014FBB700A0C3B30037
:105C500016FBB70050C0B30015FBB70080C0B300FF
:105C600017FBB7002300370050C3B30014FBB70085
:105C7000B0C3B30016FBB70040C0B30015FBB700BC
:105C8000A0C0B30017FBB7001A00370010C3B30061
:105C900014FBB700C0C3B30016FBB70030C0B3009D
:105CA00015FBB700E0C0B30017FBB70011003700C9
:105CB00060C2B30014FBB700C0C3B30016FBB7004B
:105CC00030C0B30015FBB70090C1B30017FBB7009D
:105CD00008003700C0C1B30014FBB700C0C3B30055
:105CE00016FBB70030C0B30015FBB70030C2B300DD
:105CF00017FBB7000080FA00000006000000FA0061
:105D000070F82700A0D18800803E2000B0D1880024
:105D100000712200C0D18800008F2D00D0D18800F2
:105D20000005200010D288000000EB0020D288007F
:105D30000003200030D2880040FF2F0040D28800AE
:105D40000080FA00000006001200FA008B0A07002B
:105D50002DDABF004200DD002DFAB70010168000DA
:105D6000E34060002DDABF0000C070002DFAB700DC
:105D70002DDABF000080FB00EF00600030B0210092
:105D800000804000104F78002CDABF001E40400019
:105D90002CFAB700C1A221009140780032DABF008E
:105DA00080CF500009003D002CDABF008000FB00CE
:105DB00032DABF000000FB000000EA00808F5000D4
:105DC000020034000040EB002FFAB700C1A221000E
:105DD0009140780032DABF0080CF500004003500D7
:105DE00010C0B3002FFAB7000040EB002CFAB70048
:105DF0002CDABF008000FB0032DABF000000FB009D
:105E00000000EA00808F500004003C0000C0EB005E
:105E10002FFAB7000040EB002CFAB7002FDABF00D2
:105E20000040E80063406000C600DD003CDBBF00CE
:105E3000F043B200014070003CFBB7003DDBBF0007
:105E4000664060000004E00015003A0021D58000A3
:105E50002FDABF000000FB004200DD0000804000A0
:105E600020D588000040EB002FFAB70021D5800034
:105E700000032000808F5000020034000003200047
:105E800020D5880021D5800010F82F00808F500089
:105E9000AB023D0010F82F0020D58800A802370083
:105EA0003DDBBF0066406000E24F5000BF003A009B
:105EB00040C0B30032FAB70021B021009140780011
:105EC0002FDABF0000C0400002FBB7000040EB002B
:105ED0002FFAB70002DBBF000004E00003003D0022
:105EE00002DBBF006D40400002FBB70002DBBF00D9
:105EF000EC4F50000300340002DBBF006D40500047
:105F000002FBB70040A5210021442A00130009002C
:105F10003158780002DBBF000000FB006101B900CE
:105F20005207980063079800C0002000010020007D
:105F30005E019000EE019000800F5100818F5900AA
:105F400088003E005E009000EE00900000600100BE
:105F50000C00370022003700390037003D003700C1
:105F60004100370045003700490037004D00370039
:105F70005100370055003700590037005D003700E9
:105F80006100370081A6210062452A001300090044
:105F9000B25878003CDBBF000043B200F04F500025
:105FA00067023A000040EB002EFAB7000040EB0019
:105FB00002FBB700D1B321009140780090CFB3002D
:105FC00000C060003DFBB700C1B3210091407800E4
:105FD000F0CCB30000C060003CFBB70058023700B3
:105FE00083A62100A0462A0013000900B0597800BA
:105FF0003CDBBF000043B200F04F500050023A00BB
:106000000040EB002EFAB7000040EB0002FBB700A7
:10601000D1B321009140780090CFB30000C0600060
:106020003DFBB700C1B3210091407800F0CCB30034
:1060300000C060003CFBB700C60A07004002370002
:1060400081A62100E2472A0013000900B258780017
:106050004400370083A6210020492A0013000900CC
:10606000B05978003F00370081A62100624A2A001B
:1060700013000900B25878003A00370083A62100C7
:10608000A04B2A0013000900B059780035003700F2
:1060900081A62100E24C2A0013000900B2587800C2
:1060A0003000370083A62100204E2A00130009008B
:1060B000B05978002B00370081A62100624F2A00DA
:1060C00013000900B25878002600370083A621008B
:1060D000A0502A0013000900B059780021003700B1
:1060E00081A62100E2512A0013000900B25878006D
:1060F0001C00370083A6210020532A00130009004A
:10610000B05978001700370081A6210062542A0098
:1061100013000900B25878003CDBBF000043B20016
:10612000F04F50000F003A000040EB002EFAB7008D
:106130000040EB0002FBB700D1B321009140780092
:1061400090CFB30000C060003DFBB700C1B3210099
:1061500091407800F0CCB30000C060003CFBB70079
:10616000DF04070002DBBF00E14F50000F003400E6
:106170003CDBBF000043B200F04F50000B003A0080
:10618000D1B321009140780090CFB30000C06000EF
:106190000024A0003DFBB700C1B32100914078006E
:1061A000F0CCB30000C060003CFBB7003DDBBF009B
:1061B00066406000E44F5000E1013A0002DBBF009E
:1061C0002EFAB7002EDABF008041EB00134F980083
:1061D000E94F500002003A0010C0B300104F980081
:1061E0002EDABF008040EB00014F9800EA4F5000CC
:1061F00002003A0012C0B300024F98009E4990007E
:106200008E48900001C071000080FB0030079800AC
:106210002EDABF000001EB0022079800EB4F500080
:1062200002003A001300200023079800BE009000EF
:106230002E019000028070000000E0000300320098
:1062400040C0B30032FAB7000200370020C0B300EC
:1062500032FAB7002EDABF000080FB006101B900FE
:1062600072079800030F9800B00020000100200082
:106270007E0190008E099000800F5100818F59009F
:106280009A013E007E0090008E08900000600100A0
:106290009601370095013700090037002A003700C2
:1062A0004B0037006C0037008D003700B40037001A
:1062B0008E013700D2003700EF0037005101370060
:1062C00082D280002FDABF008000FB004006200051
:1062D0000088B9000000410080D2880081D280008F
:1062E000B0D18000808F500002003D00B0D180000E
:1062F00080D2880081D28000A0D18000808F5000A1
:1063000002003400A0D1800080D2880080D28000BA
:106310003060880080D28000801F7800A0552A005D
:10632000801F780000A921002BED0700E4875700AB
:106330008041EB0072C0B300E1C0B30000A92100AE
:10634000AAFD07006901370092D280002FDABF0052
:106350008000FB00400620000088B90000004100DA
:1063600090D2880091D28000D0D18000808F5000E0
:1063700002003D00D0D1800090D2880091D28000F0
:10638000C0D18000808F500002003400C0D1800056
:1063900090D2880090D280005060880090D2800017
:1063A000801F7800A0552A00801F780000A92100D6
:1063B00009ED0700E48757008041EB0072C0B3008D
:1063C000E1C0B30000A9210088FD070047013700A4
:1063D00062D280002FDABF008000FB004006200060
:1063E0000088B9000000410060D2880061D28000BE
:1063F000B0D18000808F500002003D00B0D18000FD
:1064000060D2880061D28000A0D18000808F5000CF
:1064100002003400A0D1800060D2880060D28000E9
:106420003060880060D28000801F7800A0552A006C
:10643000801F780000A92100E7EC0700E4875700DF
:106440008041EB0072C0B300E1C0B30000A921009D
:1064500066FD07002501370072D280002FDABF00E9
:106460008000FB00400620000088B90000004100C9
:1064700070D2880071D28000D0D18000808F50000F
:1064800002003D00D0D1800070D2880071D280001F
:10649000C0D18000808F500002003400C0D1800045
:1064A00070D2880070D280005060880070D2800066
:1064B000801F7800A0552A00801F780000A92100C5
:1064C000C5EC0700E48757008041EB0072C0B300C1
:1064D000E1C0B30000A9210044FD0700030137001B
:1064E0002FDABF008000FB0000D280000080400057
:1064F00000D2880001D2800020D28000808F50001E
:1065000002003D0020D2800000D2880001D280002D
:1065100010D28000808F50000200340010D2800022
:1065200000D2880000D28000801F7800A0552A0089
:10653000801F780000A92100A7EC0700E48757001E
:106540008041EB0072C0B300E1C0B30000A921009C
:1065500026FD070000D28000760B0700F0D18000F6
:10656000E10F500003003A0000D2800000D98800FB
:10657000DE00370000D2800010D98800DB00370031
:1065800021D980002FDABF000000FB00008040000E
:1065900020D9880021D9800040D28000808F50000F
:1065A00002003D0040D2800020D9880021D980001F
:1065B00030D28000808F50000200340030D2800042
:1065C00020D9880020D98000801F7800A0552A009B
:1065D000801F780000A921007FEC0700E4875700A6
:1065E0008041EB0072C0B300E1C0B30000A92100FC
:1065F000FEFC070020D980006C0B0700BB003700B1
:10660000B2D980002FDABF000000FB006A00B90099
:1066100000004100B0D98800B0D980000000E0003F
:1066200002003D000000EB00B0D98800B1D9800025
:10663000C0032000808F500002003400C0032000FF
:10664000B0D98800B0D98000801F7800E0552A00BA
:10665000801F780000A921005FEC0700E487570045
:106660008041EB0062C0B3008040EB0000A9210034
:10667000DEFC07009D0037004ADABF00804078004A
:106680002FDABF0000C040004AFAB7004ADABF0064
:10669000E34F50000200360030C0B3004AFAB700A2
:1066A0004ADABF000080FB00801F7800D0562A0025
:1066B000801F780000A9210047EC0700E4875700FD
:1066C0008041EB0062C0B3008040EB0000A92100D4
:1066D000C6FC07004ADABF000080FB0010079800E4
:1066E0009E009000E18F50001C0032001E019000BF
:1066F000E10F510004003C009E0190000300E00007
:1067000008003200790037001E009000E20F5000B0
:10671000200032009E009000E38F50002B003200DA
:106720007200370002A92100D3572A00080009008F
:10673000335978008041EB0072C0B3008040EB0019
:1067400000A92100A9FC07000040EB0028FD07007C
:106750000040EB00BD0B07006400370000A92100DA
:1067600061582A0008000900315878008041EB0088
:1067700072C0B3008040EB0000A921009BFC070021
:1067800010C0B3001AFD070010C0B300AF0B070024
:106790005600370002A92100F3582A000900090019
:1067A000335978008041EB0072C0B3008040EB00A9
:1067B00000A921008DFC070020C0B3000CFD0700DC
:1067C00020C0B300A10B07004800370000A921003A
:1067D00091592A0009000900315878008041EB00E6
:1067E00072C0B3008040EB0000A921007FFC0700CD
:1067F00030C0B300FEFC070030C0B300930B0700AD
:106800003A0037002FDABF000000FB006A00B90031
:106810008040780031DBBF0000C0400031FBB70092
:1068200031DBBF000004E00002003D000040EB004F
:1068300031FBB70011B32100914078003ADBBF0073
:1068400080CF5000020034003ADBBF0031FBB700BC
:1068500031DBBF000000FB00801F7800305A2A00A7
:10686000801F780000A92100DBEB0700E4875700B8
:106870008041EB0062C0B3008040EB0000A9210022
:106880005AFC070031DBBF0038FBB70031DBBF002B
:106890000004E00003003A001FE1A900C302A900C0
:1068A0001200370011B321009140780040C6B300B8
:1068B00080CF500003003A001FE1A900C302A800E6
:1068C0000A0037001FE1A80031DBBF000000FB0019
:1068D000CF80DE004BE8070002002000030F2400F9
:1068E000D1E8070004E90700E00888003CDBBF00AE
:1068F0000043B200F04F50000F003A000040EB00A0
:106900002EFAB7000040EB0002FBB700D1B3210024
:106910009140780090CFB30000C060000014A00048
:106920003DFBB700C1B3210091407800F0CCB3002B
:1069300000C060003CFBB7000040EB002FFAB7003E
:106940000080FA00000006003000FA00881F78007E
:106950000000200080007800805B2A0000017800A1
:106960008101780001E023007000200043EB070064
:1069700001E02300700020007CEB07000000EB002A
:10698000000F7800D9003700F00320009E0F1000A0
:1069900024003C009E017800F00320001E005000FF
:1069A000C200DD0000E023000080400010017800FC
:1069B000F00320001E005000C200DD0000E02300B4
:1069C00000804000100078000090B90000027800BC
:1069D000F00320001E0050004200DD008080E8002F
:1069E00000E023000080400010017800F003200048
:1069F0001E0050004200DD008080E80000E023001F
:106A000000804000100078000090B90000004200B3
:106A10000001780083804100C08221000080400096
:106A2000020878001E007800701798001E00780099
:106A300080004000C08221000080400010047800E7
:106A40006140B900EFE70700501798006117980000
:106A50000800E00007003D00020020000378240049
:106A60005E109000EE10900012E80700501798009A
:106A70006117980012408500234085005E10900049
:106A8000EE10900068E80700301798004117980052
:106A900012408500234085000000200001F82300FB
:106AA00003E8070010179800211798001E007800CF
:106AB00080004000C0722100008040001004780077
:106AC0006140B900CFE70700700F980001179800E8
:106AD0000800E00007003D000200200003782400C9
:106AE0007E0890008E109000F2E70700700F98006B
:106AF000011798007E0990008E1190001E109000E2
:106B0000AE10900048E807000001BE003E10900063
:106B1000CE109000E7E7070077E807000001780053
:106B2000FE119000FE11900083804100C072210090
:106B30000080400002087800F00320009E0F100043
:106B4000690034009E017800F00B20001E00500008
:106B5000C200DD0000E0230000804000100178004A
:106B6000F00B20001E005000C200DD0000E02300FA
:106B700000804000100078000090B900000278000A
:106B8000F00B20001E0050004200DD008080E80075
:106B900000E023000080400010017800F00B20008E
:106BA0001E0050004200DD008080E80000E023006D
:106BB00000804000100078000090B9000000420002
:106BC0000001780083804100C082210000804000E5
:106BD000020878001E007800600F98001E00780000
:106BE00080004000C0822100008040001004780036
:106BF0006140B90083E70700400F9800510F9800EB
:106C00000800E00007003D00020020000378240097
:106C10004E089000DE089000A6E70700400F98009D
:106C2000510F980012408500234085004E089000C7
:106C3000DE089000FCE70700200F9800310F980055
:106C400012408500234085000000200001F8230049
:106C500097E70700000F9800110F98001E007800BA
:106C600080004000C07221000080400010047800C5
:106C70006140B90063E7070060079800710798005A
:106C80000800E00007003D00020020000378240017
:106C90006E009000FE00900086E7070060079800F5
:106CA000710798006E019000FE0190000E089000A0
:106CB0009E089000DCE707000001BE002E0890004F
:106CC000BE0890007BE707000BE807000001780092
:106CD000EE099000EE09900083804100C07221000F
:106CE00000804000020878001E0FE800F007200036
:106CF0009E0F100024FF34000000EB0030B9880024
:106D0000D2C2BF00684060000004E000080032000A
:106D1000D2C2BF00704060000004E00004003200F6
:106D20001004200040B988000006200050B98800F7
:106D3000D2C2BF00684060000004E00008003200DA
:106D4000D2C2BF00704060000004E00004003A00BE
:106D5000E001200040B98800D003200050B988002D
:106D6000D2C2BF00684060000004E00008003A00A2
:106D7000D2C2BF00704060000004E0000400320096
:106D80002004200040B988008004200050B9880009
:106D9000D2C2BF00684060000004E00008003A0072
:106DA000D2C2BF00704060000004E00004003A005E
:106DB0006003200040B98800C003200050B988005B
:106DC0000000EB00000F78004D0037001E00780037
:106DD000500798001E00780080004000C07221001B
:106DE00000804000100478006140B90005E707000A
:106DF00030079800410798000800E00007003D00B8
:106E000002002000037824003E009000CE00900095
:106E100028E70700300798004107980032408500B6
:106E2000434085003E009000CE009000CDE7070073
:106E30000200200003F823001EE707000BE807000C
:106E4000020020000304240077E70700020020006E
:106E500003F8230017E70700A7E707000001780001
:106E6000DE019000DE01900083804100C09221008D
:106E700000804000020878001E007800800040007A
:106E8000C09221000080400010007800FF0F5000E9
:106E9000060036001E00780080004000C0922100ED
:106EA00080804000F00120008008780040B9800018
:106EB0009E0F10001100340050B980009E0F10008A
:106EC0000E003D001E00780080004000C0722100CE
:106ED000008040009000780030B98000808F500022
:106EE000060036001E00780080004000C0722100BD
:106EF000008040001000780030B988001E0FE800C4
:106F0000F00720009E0F1000B0FF340038B9800059
:106F10006140B900BBE60700100798002107980000
:106F20000800E00007003D00020020000378240074
:106F30001E009000AE009000DEE6070010079800EB
:106F4000210798001E009000AE009000C7E70700E0
:106F5000324085004340850082E707001AE80700B9
:106F600030B9880041CD800060CD800000804000B5
:106F70000000D10050CD88004F0478000080FA0056
:106F8000000006000800FA00CAC2BF000080FB0033
:106F90004500DE000004A2006140600070479800D8
:106FA000CAC2BF000044B2000004E00003003A007F
:106FB00020C0B30060479800020037008040EB001B
:106FC000614798007E4190006E4090000041410072
:106FD00052479800CBC2BF00644060000004E0004C
:106FE00003003A0041C0B300414798000200370057
:106FF0000041EB0042479800DE4090004E41900077
:1070000002C04000674F6000D2C2BF00684060000D
:107010000004E0000300320040C0B300F4FA0700AF
:10702000020037004ADABF00F1FA07003DDBBF007B
:10703000664060000004E00062003A001E00FB00B1
:10704000100798009E009000E18F5000240032004D
:107050001E019000E20F51003E0032001E00900021
:107060000000E00001003200560037000000EB0095
:10707000E0D18800D2C2BF00704060000004E00090
:1070800005003A00C1A72100826B2A000400090014
:10709000B258780004003700C0A72100D16B2A0045
:1070A0000400090031587800D2C2BF006840600077
:1070B0000004E00004003200216C2A00C0A7210077
:1070C000DCE9070003003700A16C2A00C0A72100FB
:1070D000D8E907000000EB00F0D188003900370044
:1070E00010002000E0D18800D2C2BF0070406000D4
:1070F0000004E00005003A00C2A72100106D2A003C
:10710000050009003059780004003700C1A72100AC
:10711000726D2A0005000900B2587800D2C2BF0083
:10712000684060000004E00004003200216C2A0086
:10713000C0A72100BFE9070003003700A16C2A00A7
:10714000C0A72100BBE9070010002000F0D1880093
:107150001C00370010002000E0D18800D2C2BF0020
:10716000704060000004E00005003A00C0A7210064
:10717000D16D2A000500090031587800040037005D
:10718000C2A72100306E2A0005000900305978009E
:10719000D2C2BF00684060000004E000040032007A
:1071A000216C2A00C0A72100A2E9070003003700D4
:1071B000A16C2A00C0A721009EE907000000EB0097
:1071C000F0D18800000000000080FA0000000600F6
:1071D0000200FA00CAC2BF00684060000004E0007C
:1071E0000E003A00CAE2A900E0D180000000E000F1
:1071F00005003A002000200050D988000000EB0074
:1072000030D98800080037000000EB0050D9880012
:107210001000200030D98800030037001000200043
:1072200050D98800CAE2A800F0D18000E10F5000D8
:1072300013003A00120020008000EB000003200041
:10724000B604070000000000020420003103200003
:1072500000032000B10407000000000000D98000F6
:1072600000D28800CAC2BF00684060000004E0008D
:1072700015003A0000D280002E08070012003700E7
:10728000120020008000EB0000032000A304070090
:10729000000000000001EB0031032000000320008B
:1072A0009E0407000000000010D9800000D2880072
:1072B000CAC2BF00684060000004E00002003A005B
:1072C00000D280001B08070050D98000000F780012
:1072D0001E007800E10F50002F0032001E007800E1
:1072E000E20F5000560032001E0078000000E0005F
:1072F000010032006D00370000042000E3070700A2
:10730000120020008000EB0000032000830407002F
:10731000000000000001EB004103200000032000FA
:107320007E040700000000000001EB007103200054
:107330000003200079040700000000000000EB00BB
:107340001A0807000000EB003B080700C0002000FF
:10735000E3070700120020008000EB00000320007C
:107360006E04070000000000C2002000410320005E
:1073700000032000690407000000000000D2800024
:10738000EC07070060D280003060880070D2800077
:10739000506088004500370000042000BB0707004C
:1073A00000042000CE070700120020008000EB0040
:1073B0000003200059040700000000000001EB005A
:1073C00041032000000320005404070000000000D7
:1073D0000001EB0071032000000320004F040700B0
:1073E00000000000020320004103200000032000F1
:1073F0004A0407000000000002032000710320007F
:1074000000032000450407000000000020D5800094
:10741000E607070040D58000C6070700C0FE2F0022
:1074200005080700600020009807070080D2800050
:107430003060880090D28000506088001B003700C8
:107440000004200091070700120020008000EB00DC
:107450000003200031040700000000000001EB00E1
:1074600041032000000320002C040700000000005E
:107470000001EB0071032000000320002704070037
:107480000000000020D98000C8070700800120000C
:10749000930707000000EB007C07070060D2800024
:1074A0003060880070D2800050608800D2C2BF0077
:1074B000704060000004E000030032000080EB0038
:1074C00040D98800020037001000200040D9880011
:1074D000160007009660A8000080FA000000060071
:1074E0000000FA000000240060D288000000EB00D9
:1074F00070D288000000240080D288000000EB00D9
:1075000090D288000000EB0000D988000000EB005A
:1075100010D988000000EB0020D988000000EB00A3
:1075200020D588000080FA00000006000000FA0064
:10753000D2C2BF000080FB004400DE000004A200B5
:107540006140600061406000614060006140600037
:107550004201DD00212D200091407800B0CFB30022
:1075600000C0600002407000D2E2B700F0D180009D
:1075700061406000C700DD00C2C2BF000074A1000E
:1075800001407000C2E2B700CAC2BF000080FB0029
:107590004300DE0061406000614060004201DD00A8
:1075A000312C200091407800B0CFB30000C06000C3
:1075B00002407000C3E2B7000080FA00000006003D
:1075C0000000FA00CA82A900CA82A8000001EB00EC
:1075D0008000EB0000032000D00307000000000043
:1075E000120020001100200000032000CB03070040
:1075F00000000000120020008000EB0000032000CB
:10760000C6030700820020001100200000032000B4
:10761000C203070012002000210020000003200008
:10762000BE0307000001EB008000EB000003200018
:10763000BA030700D2042000B1012000000320009B
:10764000B6030700320020004100200000032000A4
:10765000B203070082002000610020000003200028
:10766000AE0307007200200071002000000320001C
:10767000AA03070002082000810020000003200068
:10768000A6030700020A2000E101200000032000F9
:10769000A20307001209200051002000000320006F
:1076A0009E03070022002000D100200000032000DC
:1076B0009A0307000001EB00E10020000003200016
:1076C000960307000208200041012000000320006B
:1076D0009203070082082000B10020000003200070
:1076E0008E03070022082000C100200000032000B4
:1076F0008A030700820820002101200000032000E7
:1077000086030700820820003101200000032000CA
:1077100082030700820020008000EB0000032000AD
:107720007E03070000000000920720008101200076
:10773000000320007903070000000000320A200047
:1077400091012000000320007403070000000000E6
:10775000D2002000A1012000000320006F030700D9
:107760000000000062082000C1012000000320008A
:107770006A03070000000000C2052000D1012000BC
:10778000000320006503070000000000320F200006
:10779000E10120000003200060030700000000005A
:1077A0003207200001022000000320005B030700D5
:1077B00000000000620420001102200000032000ED
:1077C0005603070000000000B20120002102200043
:1077D0000003200051030700000000009200200079
:1077E0008000EB00000320004C03070000000000B5
:1077F0009207200001022000000320004703070039
:1078000000000000320A20001102200000032000C6
:107810004203070000000000D200200021022000E7
:10782000000320003D030700000000006208200064
:107830004102200000032000380307000000000080
:10784000C20520005102200000032000330307007E
:1078500000000000320F2000610220000003200021
:107860002E030700000000003207200081022000E4
:10787000000320002903070000000000620420002C
:1078800091022000000320002403070000000000F4
:10789000B2012000A1022000000320001F03070006
:1078A000000000000001EB008000EB00000320005E
:1078B0001A0307000000000022002000D10320006E
:1078C0000003200015030700000000003D09070029
:1078D0007D090700BD090700FD0907007A070700B9
:1078E000120020008000EB00000320000B030700C3
:1078F0000000000042062000D10320000003200009
:1079000006030700000000000001EB00310020002A
:107910000003200001030700000000000001EB004D
:107920004100200000032000FC02070000000000CE
:10793000120020008000EB0000032000F702070087
:107940000000000082002000C10020000003200091
:10795000F20207000000000082002000D100200099
:1079600000032000ED02070000000000820020005C
:10797000E100200000032000E80207008200200050
:10798000F100200000032000E40207000001EB00EA
:107990008000EB0000032000E00207000000000070
:1079A000220020000104200000032000DB02070069
:1079B000000000000001EB00110420000003200083
:1079C000D602070000000000420D2000F103200055
:1079D00000032000D1020700000000001200200078
:1079E0008000EB0000032000CC0207000000000034
:1079F000A20020000101200000032000C7020700B0
:107A000000000000A200200011012000000320005F
:107A1000C2020700000000000001EB00210120006D
:107A200000032000BD020700000000000001EB0081
:107A30003101200000032000B80207000000000010
:107A4000C20320009100200000032000B3020700C1
:107A5000120020008000EB0000032000AF020700AE
:107A6000000000000203200041032000000320006A
:107A7000AA0207000000000002032000710320009A
:107A800000032000A50207000000000032002000D3
:107A90006103200000032000A00207000000000096
:107AA0003200200091032000000320009B02070009
:107AB0000000000082022000B1032000000320002B
:107AC000960207000000000082022000C10320008F
:107AD0000003200091020700000000000001EB00FD
:107AE0008000EB00000320008C0207000000000073
:107AF000020C20001105200000032000870207006F
:107B0000000000000001EB00210520000003200020
:107B100082020700000000000080FA00000006005A
:107B20000200FA00313A800000E02F00008060007F
:107B30006102200001007000303A8800000000005F
:107B4000417420009140780000CEB30000C0600076
:107B50000004A00044E7B7000000000044C7BF00D5
:107B6000F043B20044E7B7000000000032002000FC
:107B700081072000A009200033742000814978008B
:107B800080497800824978001200200061042000BA
:107B90007005200023742000814978008049780016
:107BA0008249780043C7BF0002C7B300824060002B
:107BB00000C3B30080CF5000FAFF3A002C83A80026
:107BC00000000000C842A8000000000068C0A80033
:107BD000000000000000EB00000F780003003700F9
:107BE000A00F0900000000001E0FE800900F200009
:107BF0009E0F1000FAFF34005000200080368800ED
:107C000010F121003035880040012000C0118800AB
:107C1000000028008011880000402000901188009A
:107C20001FE1A9001E61A9001E21A9001EC1A90013
:107C3000E111200091407800F0CCB30000C060005A
:107C40001EE1B7000000EB00A0088800E02E200035
:107C5000D0088800110B200091407800F0C8B300D4
:107C600000C0600001C5B30001407000B1E0B70082
:107C70008760A9009760A8001FE1A80021E1A90082
:107C80002021A90020C1A900011220009140780004
:107C9000F0CCB30000C0600020E1B7000000EB00B2
:107CA000C0088800210B20009140780080CFB300ED
:107CB00000C060005040B300B2E0B7008780A90068
:107CC0009780A80000000000C0032000B0D9880001
:107CD000CE01070000000000E106070000000000E0
:107CE000F0070700000000009A07070000000000EE
:107CF000AFF7070000000000B10907000000000016
:107D00002FFE070000000000F4090700000000003B
:107D1000E303070000000000EA0507000000000080
:107D2000F6F70700000000005901070000000000FE
:107D3000D00907000000000092FC070024FD0700A6
:107D40000000000000000000000A2000C0B8880009
:107D50000000EB00A0D98800CAC2BF000080FB0071
:107D60004300DE00614060000080FB0060D98800B5
:107D700010C0B30032FAB700C302A80000003700F9
:107D80003DDBBF00614060000004E00058003200AD
:107D90003D1BA9007BFC0700E4FD0700CAC2BF0031
:107DA0000080FB004300DE00614060000080FB00BB
:107DB00070D9880071D9800060D98000808F500010
:107DC0000300320002FD070070D9800060D98800EE
:107DD000D2C2BF00704060000004E0000300320027
:107DE0000080EB0040D9880002003700100020001E
:107DF00040D988003DBBA900CAC2BF0064406000F2
:107E00000004E00022003200A0B880000000E00082
:107E10001F003200A1B8800070BB2000808F50008E
:107E20000A003400C1B3210091407800F0CCB300C7
:107E300000C0600001C2B300014070003CFBB7000D
:107E40000000EB00A0B8880011003700A1B8800046
:107E500070252000808F500009003400C1B321003C
:107E600091407800F0CCB30000C060000044A00056
:107E70003CFBB7000000EB00A0B88800040037000E
:107E80003CDBBF00F1CCB300014060003CFBB7001D
:107E900031DBBF000004E00003003A001FE1A9004D
:107EA000C302A9001200370011B3210091407800ED
:107EB00040C6B30080CF500003003A001FE1A90084
:107EC000C302A8000A0037001FE1A80031DBBF0091
:107ED0000000FB00CF80DE00CAE2070002002000A5
:107EE000030F240050E3070083E30700E008880045
:107EF0003DDBBF00664060000004E00011003A0076
:107F00003CDBBF0003C3B3008340600000C2B3008A
:107F100080CF50000B003A00D1B32100914078008F
:107F200090CFB30000C060000014A0003DFBB7007C
:107F3000C1B3210091407800F0CCB30000C06000D4
:107F40003CFBB70080F707003DDBA9009660A80066
:107F500010D78000E10F500008003A00A0D980003F
:107F6000E20F500005003A0077FA07000000EB002E
:107F700010D788001000200090D9880090D9800088
:107F8000E10F50007EFF3A00A0D98000E40F5000BE
:107F90007BFF3A0021F407000000EB0090D9880035
:107FA00077FF37000000FA00889FBE0020D78000CE
:107FB000CF80DE0093E207000001BE000000200039
:107FC000A137240067E3070020E407000200200037
:107FD000031A240014E3070040D6880051D6880015
:107FE00040D6800051D680006011B8001BE4070025
:107FF0000000E00001003C000E00370040D6800089
:1080000051D6800082D6800093D68000A8E2070077
:10801000A2D68000B3D6800003E3070082D680009A
:1080200093D68000A3E2070060D6880071D688004E
:108030000D00370040D6800051D6800082D68000E7
:1080400093D680009AE20700C2D68000D3D6800083
:10805000F5E2070082D6800093D6800095E2070003
:1080600060D6880071D6880060D6800071D6800006
:10807000D5E307000001BE00F0FF2F00F1FF27004D
:10808000800F5100818F590003003A006000B80052
:1080900060D6880071D6880060D6800071D68000D6
:1080A00080D6880091D6880060D6800071D6800086
:1080B000C5E307008000780040D5800000804000C4
:1080C00040D5880040D580000000E00002003D005F
:1080D0000000EB0040D58800B1D9800040D5800079
:1080E000808F500002003D00B0D9800040D588004C
:1080F00041D5800050D58000808F500004003200B0
:1081000040D580008B04070040D5800050D5880002
:10811000403F8500513F85000004BE00F0D780003D
:10812000CF80DE0037E207000001BE000800BE007D
:108130000CE30700C5E30700020020000320240031
:10814000B9E2070020D6880031D68800F0D7800039
:10815000CF80DE002BE20700423F8500533F8500C1
:10816000BEE307000000E00001003D000E00370004
:1081700020D6800031D6800002D6800013D6800041
:108180004BE20700A2D58000B3D58000A6E207002D
:1081900002D6800013D6800046E20700E0D58800B2
:1081A000F1D588000D00370020D6800031D6800040
:1081B00002D6800013D680003DE2070062D5800021
:1081C00073D5800098E2070002D6800013D68000A5
:1081D00038E20700E0D58800F1D5880000D680009D
:1081E00011D6800078E307000001BE00F0FF2F00E9
:1081F000F1FF2700800F5100818F590003003A00E2
:108200006000B80000D6880011D68800E0D5800054
:10821000F1D580006CE307000001BE00F0FF2F00E5
:10822000F1FF2700800F5100818F590003003A00B1
:108230006000B800E0D58800F1D58800E0D5800066
:10824000F1D5800000D6880011D6880028D580009E
:10825000E0D58000F1D580005BE30700000044001A
:10826000E0D68800E1D68000F0D68000808F5000F4
:1082700004003200E0D680004C040700E0D6800005
:10828000F0D688004F04BE000080FA00000006000F
:108290000000FA0090042100E1922300A0D688009B
:1082A000B1D68800603F8500713F85000200200044
:1082B000033224005CE20700823E8500933E850085
:1082C000A8E20700A0D68800B1D68800603F8500EC
:1082D000713F8500020020000332240052E20700B3
:1082E000A23E8500B33E85009EE20700C0D688000E
:1082F000D1D68800603F8500713F850002002000D4
:108300000332240048E20700C23E8500D33E8500C8
:1083100094E2070060D5880071D58800603F850031
:10832000713F850002002000033224003EE2070076
:10833000E23E8500F33E85008AE20700A0D5880072
:10834000B1D5880062D5800073D580000000200080
:1083500001F82300D6E1070080D5880091D5880078
:10836000A2D58000B3D580000000200001F82300D2
:10837000CFE10700C0D58800D1D58800003F850037
:10838000113F8500623F8500733F850075E207005D
:108390000DE30700D0D78800203F8500313F8500DE
:1083A000623F8500733F85006EE2070006E3070029
:1083B000C0D788000000EB00F0D788000000EB0079
:1083C00000D888006000B800E0D58800F1D58800AA
:1083D0006000B80000D6880011D688000000EB00CD
:1083E00020D788000000EB0030D788000000EB00A9
:1083F00030D58800B0D9800040D5880040D58000B5
:1084000050D588000080FA00000006000000FA0045
:108410000000EB00001088000000EB001010880046
:108420000000EB00501088000000EB006010880096
:1084300000042000201088000602A90000000000AF
:108440000622A900000000000642A900000000006A
:108450000662A900000000000682A90000000000DA
:1084600006A2A9000000000006C2A900000000004A
:1084700006E2A900000000000702A90000000000B9
:108480000722A900000000000742A9000000000028
:108490000762A900000000000782A9000000000098
:1084A00007A2A9000000000007E2A80000000000E9
:1084B0000802A900000000000822A9000000000036
:1084C0000842A900000000000862A90000000000A6
:1084D0000882A9000000000008A2A9000000000016
:1084E00008C2A9000000000008E2A9000000000086
:1084F0000902A900000000000922A90000000000F4
:108500000942A9000000000009C2A9000000000003
:1085100009E2A9000080FA00000006000400FA0049
:10852000004F780011479800224798000602A800E3
:10853000301080007F0060000000E000FCFF3A0087
:108540001E80FB001010880009C2BF000044B2006A
:108550000004E000FCFF3A001E4090000080FB0099
:108560001010880009C2BF000044B2000004E000FF
:10857000FCFF3A002E4090000080FB0010108800A5
:1085800009C2BF000044B2000004E000FCFF3A0052
:108590000642A80006C2BF00644060000004E0007C
:1085A000FCFF3A000080FA00000006000400FA0018
:1085B000000F7800214798000602A80030108000C4
:1085C0007F0060000000E000FCFF3A00000A20008D
:1085D0001010880009C2BF000044B2000004E0008F
:1085E000FCFF3A001E0078004880DE001010880072
:1085F00009C2BF000044B2000004E000FCFF3A00E2
:108600001E0078001010880009C2BF000044B200AC
:108610000004E000FCFF3A002E4090000000FB0048
:108620001010880009C2BF000044B2000004E0003E
:10863000FCFF3A000642A80006C2BF00644060008A
:108640000004E000FCFF3A00570007000080FA0039
:10865000000006000400FA00100798000602A800B7
:1086600006C2BF00614060000004E000FCFF3A0069
:10867000000A20001010880009C2BF000044B200A8
:108680000004E000FCFF3A001E0090004880DE007D
:108690001010880009C2BF000044B2000004E000CE
:1086A000FCFF3A001E0090001010880009C2BF00B5
:1086B0000044B2000004E000FCFF3A000622A800DB
:1086C00006C2BF00624060000004E000FCFF3A0008
:1086D000100A20001010880009C2BF000044B20038
:1086E0000004E000FCFF3A0009C2BF0001C8B3006B
:1086F000014060000004E000FBFF3A000662A800B1
:1087000006C2BF00684060000004E000FCFF3A00C1
:1087100000108000004F780006A2A8000682A80082
:1087200006C2BF00704060000004E000FCFF3A0099
:108730000642A80006C2BF00644060000004E000DA
:10874000FCFF3A001E00FB000080FA00000006005B
:108750000200FA000000EB00000F78000200370072
:10876000000000001E0FE800700020009E0F1000A7
:10877000FBFF34000080FA00000006000200FA004F
:108780000000EB00000F780002003700000000003E
:108790001E0FE800F0F920009E0F1000FBFF3400D0
:1087A0000080FA00000006000200FA000000EB0062
:1087B000000F780002003700F0FF07001E0FE800EE
:1087C000100320009E0F1000FBFF34000080FA0011
:1087D000000006000200FA000000EB00000F780025
:1087E00002003700E5FF07001E0FE800900F200091
:1087F0009E0F1000FBFF34000080FA00000006000E
:108800003600F800809FBE00829FBE00849FBE009D
:10881000869FBE00889FBE000200FA008B80A900E0
:10882000CAC2BF00644060000004E00003003A00D8
:10883000A0B880000000E800A0B8880000688000B0
:108840000000E800006888000168800080252000A2
:10885000808F500003003A003D1BA8000000EB0091
:108860000068880050D98000000F78001E01780051
:10887000E10F5100150032001E007800E20F500099
:10888000460032001E0178000200E00001003200C4
:10889000A8003700801480002060880020608000DD
:1088A000906088009014800000B988004D04070093
:1088B00040608000C0148800B160800040D9800012
:1088C0000088B900D01488009A0037009014800006
:1088D000E0B8880080148000F0B88800C0B880003C
:1088E000E2B880008000400040D1200000804000BD
:1088F00002087800C0B88000F2B880008000400014
:1089000040F920000080400002087800C0B88000D4
:108910000000E800C0B88800C1B88000000A20004C
:10892000808F500005003A0010002000D0B8880069
:108930000000EB00B0B888009460A800C1B88000C7
:1089400000142000808F500007003A000000EB0068
:10895000C0B8880010002000D0B88800000A2000AD
:10896000B0B888009460A800C0B8800080004000C3
:10897000402121000080400010007800C0148800D1
:10898000C0B88000800040004049210000804000C5
:1089900010007800D014880066003700116880004D
:1089A000A03F8500008040001068880010688000AB
:1089B00002002100110009000200D8008000FD0023
:1089C00010688800D2C2BF000042B2000004E0007C
:1089D000040032006000B80010B9880021B9880096
:1089E00004003700F03F85000140850010B9880081
:1089F00021B9880010B9800021B980004268800048
:108A0000536880002AE00700B23F8500C33F85001D
:108A100085E007000004BE00D03F8500E13F8500EF
:108A200042688000536880007FE007000001BE00BC
:108A30000800BE001FE00700206888003168880039
:108A40002068800031688000826880009368800020
:108A500017E00700B23F8500C33F850072E00700C2
:108A60000004BE00D03F8500E13F850082688000A1
:108A7000936880006CE007000001BE000800BE00A3
:108A80000CE007006068880071688800206880003A
:108A900031688000406888005168880080688000E4
:108AA0009168800080688800916888008014800048
:108AB00000B988009014800000B9880060688000C8
:108AC0007168800040E107000004BE00106880006B
:108AD000C00507006103B90088007800060078002F
:108AE000000AB80007C0B900050178000001410084
:108AF00009B0B90000014100820278004129DD007F
:108B00004F20DE0000007100CFA8DE00206088004A
:108B10002060800090608800B20307004060800001
:108B2000C0148800B160800040D980000088B9007E
:108B3000D01488000080FA004F04BE004F03BE002E
:108B40004F02BE004F01BE004F00BE003600F900CC
:108B5000004006000000FA00C1A421009140780006
:108B60000000EB0091FE0700D1A4210091407800A5
:108B7000100020008DFE0700E1A421009140780044
:108B80002000200089FE0700F1A421009140780018
:108B90003000200085FE070001A5210091407800EB
:108BA0004000200081FE070011A5210091407800BF
:108BB000500020007DFE070021A521009140780093
:108BC0006000200079FE070031A521009140780067
:108BD0007000200075FE070001B22100914078006E
:108BE0008000200071FE070011B221009140780042
:108BF000900020006DFE070021B221009140780016
:108C0000A000200069FE070031B2210091407800E9
:108C1000B000200065FE070041B2210091407800BD
:108C2000C000200061FE070051B221009140780091
:108C3000D00020005DFE070041AA2100914078008D
:108C4000E000200059FE070051AA21009140780061
:108C5000F000200055FE070061B32100914078002C
:108C60000001200051FE070071B3210091407800FF
:108C7000100120004DFE07004ADABF008040780056
:108C80002001200049FE070081B3210091407800B7
:108C90003001200045FE07000080FA0000000600B9
:108CA0000000FA000000EB006AFE07004CFAB70073
:108CB0001000200067FE07004DFAB700000000001A
:108CC000000000002000200062FE07004EFAB700FE
:108CD000300020005FFE07004FFAB70000000000E0
:108CE00000000000400020005AFE070050FAB700C4
:108CF0005000200057FE070051FAB70000000000A6
:108D0000000000006000200052FE070052FAB70089
:108D1000700020004FFE070053FAB700000000006B
:108D200000000000800020004AFE070020FBB70082
:108D30009000200047FE070021FBB7000000000064
:108D400000000000A000200042FE070022FBB70048
:108D5000B00020003FFE070023FBB700000000002A
:108D600000000000C00020003AFE070024FBB7000E
:108D7000D000200037FE070025FBB70000000000F0
:108D800000000000E000200032FE0700A4FAB70057
:108D9000F00020002FFE0700A5FAB7000000000039
:108DA00000000000000120002AFE070036FBB7008B
:108DB0001001200027FE070037FBB700200120002C
:108DC00024FE07004AFAB7003001200021FE070008
:108DD00038FBB70038DBBF0031FBB70000000000F4
:108DE000000000000080FA0000000600361B0000B2
:108DF0000400000000000000004300000004000028
:108E00000000000000080000000500000000000055
:108E1000141B00000C000000000000003A1B0000C2
:108E20000200000002000000640000002C1B000093
:108E30000A00000000000000003E000000020000E8
:108E400000000000261700000603000000000000DC
:108E5000E01A00002200000000000000A41A000038
:108E60003C00000000000000000D0000260A000089
:108E700000000000201B00000C00000000000000AB
:108E80003C1B00000200000000000000021B00006C
:108E9000120000000200000000000100FF00FF00BF
:108EA0000000010001000000FF00FF0001000000C1
:108EB0002C1A000078000000000000003E1B00009B
:108EC000020000000000000000470000A0000000B9
:108ED00002000000010000000000000000000A0085
:108EE000000000000000000000640000000000001E
:108EF00000000000E8030000000000000000100077
:108F0000270000000000000000A086000100000013
:108F10000000000040420F00000000000000800040
:108F200096980000000000000000E100F505000038
:108F30000000000000CA9A003B0000000000000092
:108F4000E40B5400020000000000E800764817001F
:108F5000000000000010A500D4E8000000000000A0
:108F6000A0724E0018090000000040007A10F300C3
:108F70005A0000000080C600A47E8D00030000009F
:108F800000C16F00F2862300000000008A5D7800B7
:108F90004563010000006400A7B3B600E00D0000C7
:108FA00000E889000423C7008A000000A0470000F1
:108FB0002A00000002000000286E75006C6C290079
:108FC0000030310032333400353637003839410053
:108FD000424344004546000030313200333435000E
:108FE000363738003961620063646500660000004E
:108FF000CA4700002600000002000000CC47F20033
:1090000047000000F2470900000000000200F000E5
:1090100047000000F04706000201000000000000C9
:109020000000000000000600020200000000000036
:10903000F04700000600000000000000F6470000B6
:10904000020000000200000001000000000000001B
:109050000A00FA000000EB002007980085003700A6
:10906000B1B880002E0090000080400080004000D9
:1090700040D1200000804000900078001107980047
:109080001E00900020608800B1B880002E00900083
:10909000008040008000400040F920000080400037
:1090A000100F78009E0078009160880070D78000D3
:1090B000006188004B020700B160800040D9800049
:1090C0000088B900B060880041608000B060800016
:1090D0000080400070D78800D2C2BF0068406000A6
:1090E0000004E0000300320070D7800050D78800F1
:1090F000020037001061800050D78800B1B88000AE
:109100002E0090000080400052D780008000400078
:10911000402121000080400002087800B1B88000A2
:109120002E0090000080400052D780008000400058
:1091300040492100008040000208780010D78000DC
:109140000000E00018003A0000D780006260800054
:10915000C200DD0000E0230000804000020878002B
:1091600000D78000D26080004200DD008080E800EF
:1091700000E02300008040000208780000D7800053
:109180000000E80000D7880001D780000008200018
:10919000808F500004003A000000EB0000D78800E8
:1091A0001000200010D788001E0090004007980093
:1091B000CE0090000100E00003003D004E00900052
:1091C0000000EA0040079800CE00900041D78800D8
:1091D00041D7800030D7800000805000D2D7800077
:1091E000110009000200D8008000780030D780000C
:1091F0000080400020D7880020D7800030D788002A
:1092000020D7800080D7880050D780003007980092
:109210003E0090000000E00003003D00BE00900012
:109220008100EA00310798003E009000E0D78800F6
:10923000E1D7800000D8800000805000C2D78000B5
:10924000110009000200D8008000780000D88000DA
:1092500000804000F0D78800F0D7800000D8880058
:10926000F0D7800090D788002E0090000000E80022
:1092700020079800AE009000F0092000808F500079
:1092800077FF34000080FA00000006000200FA00B8
:10929000000F780012C0B3008040EB0000C3B300A1
:1092A0009EFC0700000000001E00780000417800CE
:1092B00001C1B30000C3B30098FC07000000000028
:1092C0001E0078000041780011C1B30000C3B30054
:1092D00092FC0700000000000080FA000000060079
:1092E0000200FA00000F780012C0B3008040EB00CB
:1092F00000C3B30089FC0700000000001E007800D6
:109300000041780021C1B30000C3B30083FC070013
:10931000000000001E0078000041780031C1B30059
:1093200000C3B3007DFC0700000000000080FA00CD
:10933000000006000200FA00000F78001E00E000A6
:1093400002003D000000EB00000F7800F005200057
:109350009E0F100002003400F0052000000F78007E
:1093600012C0B3008040EB0000C3B3006BFC0700E9
:10937000000000001E00780000417800B1C3B30077
:1093800000C3B30065FC0700000000001E00780069
:1093900000417800C1C3B30000C3B3005FFC070005
:1093A000000000000080FA00000006000200FA0041
:1093B000000F7800000320009E0F10000200340010
:1093C00000032000000F780010F82F009E0F1000FF
:1093D00002003D0010F82F00000F78001E00E00092
:1093E00002003D00001020001E0F40000041EB0075
:1093F0008040EB0000C3B30048FC07000000000001
:109400001E0078000041780011C4B30000C3B3000F
:1094100042FC0700000000001E00780000417800B8
:1094200021C4B30000C3B3003CFC070000000000EF
:109430000080FA00000006000200FA00000F780029
:10944000800220009E0F10000200340080022000E5
:10945000000F780080FE2F009E0F100002003D00DC
:1094600080FE2F00000F78001E00E00002003D008B
:10947000F00720001E0F40000041EB008040EB0091
:1094800000C3B30025FC0700000000001E007800A8
:109490000041780031C5B30000C3B3001FFC0700D2
:1094A000000000001E0078000041780041C5B300B4
:1094B00000C3B30019FC0700000000000080FA00A0
:1094C000000006000200FA000008200010308A00A8
:1094D000008020001060880010608000F00FB00055
:1094E0000060880000302400E00FB00000308A00E7
:1094F0000008200030308A00009020008060880042
:1095000080608000F00FB000706088000040240090
:10951000E00FB00020308A000000EB00000F780060
:10952000210037001E0078008000400000802000ED
:10953000808040000000EB00800878001E01780069
:109540001E0078008000400020AB29000080400011
:10955000900178008200410000302400008040002B
:10956000030878001E007800800040000090200072
:10957000808040000000EB00800878001E01780029
:109580001E0078008000400020BB290000804000C1
:1095900090017800820041000040240000804000DB
:1095A000030878001E0FE800F00720009E0F10004F
:1095B000DCFF3400F007200050308A0000A02000BB
:1095C000F0608800F0608000D00FB000E06088009C
:1095D00000502400C00FB00040308A004ADABF00BB
:1095E0001A00070000002400A06088000080FA0034
:1095F000000006000200FA000000EB00000F7800F7
:109600000D0037001E0078008000400000A0200000
:10961000808040000000EB00800878001E00780089
:109620008000400000502400808040000000EB00DB
:10963000800878001E0FE800E00720009E0F100051
:10964000F0FF34000080FA00000006000400FA0079
:10965000204798000000EB00000F7800150037004D
:109660001E0078008000400000A0200080804000A4
:109670000000EB00800878009E0178009E007800D2
:109680002E4090000081FB006508B90002004000F8
:109690008000400020CB29000080400010017800AD
:1096A00083804100005024000080400002087800C0
:1096B0001E0FE800E00720009E0F1000E8FF3400B6
:1096C0000080FA00000006003000FA000E80E8007A
:1096D000017C2A000E00090031587800F000B1002A
:1096E00071004700117B2A000E00090031587800F4
:1096F000F000B100000220000E004000217A2A0094
:109700000E00090031587800F000B1000000EB00B5
:10971000000F780082C0B3008040EB0000C3B300AC
:109720007EFB0700000000000B0037009E00780061
:109730000E80E80000804000104178009E00780014
:1097400071004700E140780000C3B30073FB0700DD
:10975000000000001E0FE800800020009E0F100097
:10976000F2FF340092C0B3008040EB0000C3B300AE
:109770006AFB0700000000000B0037009E00780025
:109780000E80E80000804000104178009E007800C4
:1097900071004700E140780000C3B3005FFB0700A1
:1097A000000000001E0FE800E10020009E8F100066
:1097B000F2FF34000000EB00000F78000D003700CE
:1097C0009E0078000E80E800008040001041780084
:1097D0009E007800000220000E0040000080400043
:1097E0009040780000C3B3004CFB0700000000006D
:1097F0001E0FE800200020009E0F1000F0FF340034
:10980000A2C0B3008040EB0000C3B30043FB0700DD
:10981000000000000D0037009E0078000E80E80078
:1098200000804000104178009E0078000002200077
:109830000E004000008040009040780000C3B3005C
:1098400036FB0700000000001E0FE800E1002000CA
:109850009E8F1000F0FF34000080FA000000060028
:109860000000FA002D23A800000000002D43A800EE
:10987000000000002D63A800000000002D83A80058
:10988000000000002C03A800000000002C23A8000A
:10989000000000002C83A800000000002CA3A800FA
:1098A000000000002CC3A800000000002CE3A8006A
:1098B000000000002D03A80000000000C882A900DD
:1098C00000000000C8E2A90000000000C982A90051
:1098D00000000000D002A90000000000D022A80073
:1098E00000000000D042A90000000000C142A90011
:1098F00000000000C0E2A90000000000C102A900B1
:1099000000000000C082A90000000000C16C20001F
:109910009140780000CEB30000C06000D040B3009A
:10992000CCE6B70000000000116B200091407800E9
:1099300000CEB30000C06000D040B300B1E6B70075
:1099400000000000216B20009140780000CEB300A1
:1099500000C06000F040B300B2E6B70000000000B5
:10996000016B20009140780000CEB30000C0600081
:10997000E040B300B0E6B700000000006840A80077
:10998000000000006860A8000000000068C0A80097
:109990000000000068E0A8000000000069E0A800E6
:1099A000000000006A00A800000000006B00A80092
:1099B000000000006B20A800000000006B40A80021
:1099C000000000006B60A800000000006B80A80091
:1099D000000000006040A8006060A8000080FA005D
:1099E000000006004600F8004800F8004A00F800B1
:1099F0004400F8003400F8003600F800851F7800B5
:109A0000861F7800881F78008A1F7800080B2000C6
:109A10002802880088FF280038028800256080001E
:109A2000366080001301C4000000CD006060880033
:109A300025608000566080001301C4000000CD0046
:109A4000C0608800606080000880200048028800B4
:109A50000860800058028800113082008100E9000F
:109A600018608000001C7800186088000A308200AE
:109A70000218C300018009005E18C4000500CD0073
:109A80004560880095608000A66080001301C400D6
:109A90000000CD00D0608800D5608000C6608000E6
:109AA00006804200D06088000890200048028800AC
:109AB0007860800058028800313082008100E9001F
:109AC00088608000001C7800886088002A3082004E
:109AD0000218C300018009005E18C4000500CD0013
:109AE000B56088000061800008A02000480288005E
:109AF000E860800058028800513082008100E9004F
:109B0000F8608000001C7800F86088004A3082000D
:109B10000218C300018009005E18C4000000CD00D7
:109B2000106188004F0578004F0478004F037800DB
:109B3000CF0278003600F9003400F9004400F90043
:109B40004A00F9004800F9004600F9000000000052
:109B5000000006000000FA008040EB000040EB002F
:109B6000050007008040EB0010C0B30002000700B2
:109B70000080FA00000006000400FA002047980068
:109B800031479800D322A900000420004012880029
:109B900040C2BF00614060000004E000FCFF3200F2
:109BA00040128000004F78002E4090000080FB00A3
:109BB0004012880040C2BF00614060000004E00025
:109BC000FCFF320040128000004F78003E409000C1
:109BD0000080FB004012880040C2BF00614060006E
:109BE0000004E000FCFF320040128000004F7800CB
:109BF000D322A8000080FA00000006000400FA004A
:109C000020479800D322A90040128000004F78001E
:109C1000100420004012880040C2BF006140600074
:109C20000004E000FCFF32002E4090000080FB00AA
:109C30004012880040C2BF00614060000004E000A4
:109C4000FCFF32000000EB004012880040C2BF0061
:109C5000614060000004E000FCFF32004012800020
:109C6000004F780040C2BF00614060000004E00087
:109C7000FCFF32000000EB004012880040C2BF0031
:109C8000614060000004E000FCFF320040128000F0
:109C9000004F7800D322A8001E80FB000080FA004D
:109CA000000006000000FA00D0C2A9000000000079
:109CB000D102A90000000000D122A900000000008C
:109CC000816A20009140780000CEB30000C060009F
:109CD0007041B300A8E6B70000000000616D2000ED
:109CE0009140780000CEB30000C060007040B30027
:109CF000D6E6B70000000000816D2000914078009A
:109D000000CEB30000C060000034A000D8E6B70069
:109D1000000000002124200091407800C0CFB30053
:109D200000C060000014A00042E2B7000000000084
:109D300042C2BF00C041B30042E2B70000000000D1
:109D400042A2A8000000000042C2A90000000000DA
:109D500042E2A900000000004302A8000000000049
:109D60004322A900000000004342A90000000000B7
:109D70004362A900000000004382A9000000000027
:109D80004422A8000000000045A2A8000000000036
:109D900045C2A9000000000045E2A9000000000043
:109DA00041A2A9000000000041E2A800000000005C
:109DB00040C2A90000000000D322A8000080FA00E1
:109DC000000006003000FA000E80E80081702A00D2
:109DD0000E00090031587800F000B1007100470012
:109DE000916F2A000E00090031587800F000B10090
:109DF000000220000E004000A16E2A000E000900A3
:109E000031587800F000B1000000EB00000F78003E
:109E100082C0B3008040EB0000C3B300BFF907006D
:109E2000000000000B0037009E0078000E80E80064
:109E300000804000104178009E00780071004700CB
:109E4000E140780000C3B300B4F90700000000004F
:109E50001E0FE800E00020009E0F1000F2FF34000B
:109E60000000EB00000F780092C0B3008040EB00D0
:109E700000C3B300A9F90700000000000D0037007F
:109E80009E0078000E80E8000080400010417800BD
:109E90009E007800000220000E004000008040007C
:109EA0009040780000C3B3009CF907000000000058
:109EB0001E0FE800E10020009E8F1000F0FF34002C
:109EC0000080FA00000006003000FA000E80E80072
:109ED00061732A000E00090031587800F000B100CB
:109EE0007100470071722A000E0009003158780095
:109EF000F000B100000220000E00400081712A0035
:109F00000E00090031587800F000B1000000EB00AD
:109F1000000F780082C0B3008040EB0000C3B300A4
:109F20007EF90700000000000B0037009E0078005B
:109F30000E80E80000804000104178009E0078000C
:109F400071004700E140780000C3B30073F90700D7
:109F5000000000001E0FE800E00020009E0F10002F
:109F6000F2FF34000000EB00000F780092C0B30055
:109F70008040EB0000C3B30068F907000000000058
:109F80000D0037009E0078000E80E8000080400041
:109F9000104178009E007800000220000E00400072
:109FA000008040009040780000C3B3005BF90700D8
:109FB000000000001E0FE800E10020009E8F10004E
:109FC000F0FF34000080FA00000006003000FA00C4
:109FD0000E80E80041762A000E0009003158780012
:109FE000F000B1007100470051752A000E00090011
:109FF00031587800F000B100000220000E0040004F
:10A0000061742A000E00090031587800F000B10098
:10A010000000EB00000F780082C0B3008040EB002E
:10A0200000C3B3003DF90700000000000B0037003B
:10A030009E0078000E80E80000804000104178000B
:10A040009E00780071004700E140780000C3B30033
:10A0500032F90700000000001E0FE800E0002000B9
:10A060009E0F1000F2FF34000000EB00000F78009C
:10A0700092C0B3008040EB0000C3B30027F9070093
:10A08000000000000D0037009E0078000E80E80000
:10A0900000804000104178009E00780000022000FF
:10A0A0000E004000008040009040780000C3B300E4
:10A0B0001AF90700000000001E0FE800E100200070
:10A0C0009E8F1000F0FF34000080FA0000000600B0
:10A0D0003000FA000E80E80021792A000E00090005
:10A0E00031587800F000B1007100470031782A0043
:10A0F0000E00090031587800F000B1000002200085
:10A100000E00400041772A000E0009003158780007
:10A11000F000B1000000EB00000F780082C0B30037
:10A120008040EB0000C3B300FCF807000000000013
:10A130000B0037009E0078000E80E8000080400091
:10A14000104178009E00780071004700E1407800DF
:10A1500000C3B300F1F80700000000001E0FE80084
:10A16000E00020009E0F1000F2FF34000000EB0022
:10A17000000F780092C0B3008040EB0000C3B30032
:10A18000E6F80700000000000D0037009E00780090
:10A190000E80E80000804000104178009E007800AA
:10A1A000000220000E004000008040009040780037
:10A1B00000C3B300D9F80700000000001E0FE8003C
:10A1C000E10020009E8F1000F0FF34000080FA00B4
:10A1D000000006000A00FA00300798003E009000D8
:10A1E00002402000110009000200D800200798005A
:10A1F0003E00900002402000110009000200D8003B
:10A200008000FD00100798002E0090004007980085
:10A210004E009000E10F5000140032004E009000FC
:10A22000E10F500004003C004E0090000000E000F0
:10A2300008003200240037004E009000E20F50006A
:10A24000120032004E009000E30F50001600320062
:10A250001D0037001E00900080004000002B2900E8
:10A2600000804000100F78001700370001402000E8
:10A270001E0090000080500080004000002B29004C
:10A2800000804000100F78000F0037001E00900083
:10A2900080004000002B2900008040001000780062
:10A2A000000FEA0008003700014020001E00900067
:10A2B0000080500080004000002B290000804000FA
:10A2C00010007800000FEA001E0078000080FA00FD
:10A2D000000006003600F800809FBE00829FBE008E
:10A2E000849FBE00869FBE003400F800000020005E
:10A2F000A00188000000FA00C282A80054FB0700F9
:10A3000028F707000000EB00D0B88800A0D9800033
:10A310000000E800A0D98800A0D98000E60F500016
:10A3200002003A000000EB00A0D98800C282A90018
:10A330008460A9009460A9000080FA003400F9004C
:10A340004F03BE004F02BE004F01BE004F00BE00D3
:10A350003600F90000400600801F78003400F80045
:10A3600000002000A00188000000FA008760A9001A
:10A37000C302A8000000EB00C008880021E1A8008B
:10A380000080FA003400F9004F0078000040060019
:10A390003400F800881F780008002000A801880019
:10A3A0004F0478000000FA008780A900C302A900CA
:10A3B00021E1A9000080FA003400F9000040060005
:10A3C0000000FA000000EB00001488000000EB0021
:10A3D000C01488000000EB00D01488000000EB00DF
:10A3E000E01488000000EB00F01488008142A8000F
:10A3F0000000EB0020148800012820009140780024
:10A40000C0CFB30000C0600080E2B7008102A800A6
:10A410008122A90011148000F0E12F00008060006B
:10A4200001022000010070001014880080C2A90001
:10A4300080A2A80082C2BF00F040B30082E2B70051
:10A440003000200040148800300020006014880094
:10A45000312820009140780030CFB30000C0600068
:10A460000024A00083E2B70081E2A8000080FA0087
:10A47000000006000000FA000421A900000000000E
:10A480000441A90000000000411020009140780024
:10A49000F0CCB30000C0600004E1B7000000000091
:10A4A00004C1A9000000000005A1A900A580A90021
:10A4B000A5A0A900A5C0A8002000200010088800C1
:10A4C00005E1A8008460A9000080FA0000000600F1
:10A4D0000000FA000080FA00000006000000FA0008
:10A4E00042C0BF007F40600042E0B70081E0A900A9
:10A4F000210C20009140780080CFB30000C06000A4
:10A500006040B300C2E0B7008B80A9009B80A80028
:10A51000D10A200091407800F0C8B30000C060006C
:10A5200001C2B30001407000ADE0B7008660A90031
:10A530009660A8000080FA00000006003400F800D1
:10A54000881F780008002000A80188004F047800C8
:10A550000000FA008660A9009660A9003DDBA80013
:10A560000080FA003400F90000400600FFFFFF0001
:10A57000FFFFFF00FFFFFF00FFFFFF00FFFFFF00E7
:10A58000FFFFFF00FFFFFF00FFFFFF00FFFFFF00D7
:10A59000FFFFFF00FFFFFF00FFFFFF00FFFFFF00C7
:10A5A000FFFFFF00FFFFFF00FFFFFF00FFFFFF00B7
:020000040002F8
:10A000000A0000004FE020000E7F24000E018800AF
:10A01000000000000C000700404D2500110020004A
:10A0200011000700000020000000E00002003200E4
:10A030000000020000000000925002000100000039
:10A040000040DA000000FE004440A90000002000AB
:10A050000000E0000300320000002000A0018800A2
:10A060004440A800000006009101880080007800AC
:10A070000000EB0015003700E280400032A0B40081
:10A080009101BA00E280400032A0B4009102BA000F
:10A09000E280400032A0B4000002EB00472BDE005B
:10A0A000F507B200602CE10004003A000059EB0013
:10A0B0008301E900FDFF3E00040037006128E10054
:10A0C000010032000082EB00040007001101BA0019
:10A0D0000200E000E8FF3A00000006003159BA0033
:10A0E0008301E9000C0032002159BA008301E90024
:10A0F000080032000400E00003003A00E280400063
:10A1000032A0B400F5FF370011D9BA008301E9008D
:10A11000FAFF3A008100E800E180400032A0B4007C
:10A12000000006002C00FA00313A800000E02F0009
:10A13000008060006102200001007000303A880059
:10A1400000000000417420009140780000CEB30070
:10A1500000C060000004A00044E7B7000000000059
:10A1600044C7BF00F043B20044E7B700000000005E
:10A170003200200081072000A00920003374200055
:10A1800081497800804978008249780012002000D7
:10A1900061042000700520002374200081497800AC
:10A1A000804978008249780043C7BF0002C7B300E6
:10A1B0008240600000C3B30080CF5000FAFF3A0035
:10A1C00040A7A9000000000042C7BF000042B20043
:10A1D0000004E000FCFF3200000000002C83A80017
:10A1E000000000002CC3A800000000002CE3A80021
:10A1F00000000000C842A8000000000068C0A800DD
:10A20000000000000000EB00300798000500370058
:10A21000A00F0900000000003E0090000000E800D0
:10A2200030079800BE009000900F2000808F5000F3
:10A23000F7FF3400D022A8005000200080368800AC
:10A2400010F121003035880040012000C011880045
:10A250000000280080118800004020009011880034
:10A2600000002500110020004007980051079800C9
:10A27000CE0090005E009000B501070060079800D6
:10A28000710798004E4890000004E00001003A0079
:10A29000B3010700CAC2BF00644060000004E000D0
:10A2A00001003200AE0107001061A8008500A9007E
:10A2B0009500A9004E4890000003FB00CFB3DE00DC
:10A2C0008600780000A02500000AB80020262000A3
:10A2D00000B0B900050178000001410000A0250090
:10A2E00000B8B900000141008202780064079800BC
:10A2F000750798007E009000700888006E0090003E
:10A300006008880011E1A8000000370070004700D5
:10A31000BF0007000E5090000000FB00501798008F
:10A32000DE119000E38F5100260032005E10900095
:10A33000E30F500007003C005E1190000200E000B7
:10A34000AE003200DE119000E28F51000B003200AF
:10A35000AC0037005E109000E80F50007A00320029
:10A360005E119000E90F51003A003200DE119000BA
:10A37000E78F510050003200A20037007200470002
:10A38000A3000700720047000000E800A0000700DB
:10A39000720047000080E8009D0007000040EB00CD
:10A3A000505798001E099000AE09900000802000D0
:10A3B000B70007000160200000802000DA000700DD
:10A3C000D2FF370076004700910007007600470073
:10A3D0000000E8008E000700760047000080E800DB
:10A3E0008B0007000040EB00105F98000000EB00BE
:10A3F00020079800080037002E00900080007800A9
:10A400000080200000804000810007002E009000A6
:10A410000000E80020079800AE009000F05F2000E8
:10A42000808F5000F4FF3400BE0890004E0890006A
:10A43000220424004D0107003E099000CE0990003F
:10A4400000802000D400070010C0B300C80007003F
:10A45000AEFF370000002000F10F2000500F9800E1
:10A46000610F9800DE0890006E0890003801070028
:10A47000700F9800011798007E00470041002000EF
:10A48000A900070020002000F10F2000500F9800C5
:10A49000610F9800DE0890006E0890002C01070004
:10A4A000700F9800011798007E00470041002000BF
:10A4B0009D00070095FF37000000EB001007980093
:10A4C0001D0037001E0090008000780000802000F2
:10A4D000808040001E0090000000E80010079800F7
:10A4E000010078004A0007001E00900080007800FC
:10A4F00000802000808040001E0090000000E800E6
:10A500001007980001007800410007001E0090002D
:10A510008000780000802000808040001E009000B5
:10A520000000E800100798000100780038000700DC
:10A5300010C0B3008E0007001E009000F70F5000FF
:10A54000E0FF340071FF37000000EB00000F7800DF
:10A5500000002000810F200010179800211798009C
:10A56000210037009E00780000802000008040001D
:10A57000104078000004E00013003A009E00E8005C
:10A580000080200000804000104078006067980044
:10A590009E80E8000080200000804000104078008D
:10A5A000706798003E1090004E1190009E10900031
:10A5B0002E1290008001780004007800E00007006F
:10A5C00000002400D30007001E007800630F400045
:10A5D0001E109000AE10900062004000E080480025
:10A5E0001017980021179800720120009E0F11008B
:10A5F000DCFF3400DA00070044FF3700D800070012
:10A6000042FF37000040EB00590007003FFF3700D2
:10A610000200FA00000F78000000370085C0BF007C
:10A62000614060000004E000040032009E007800F9
:10A630000040EB00804878001300370032C2BF00B2
:10A64000644060000004E000F4FF3A0032C2BF0042
:10A65000624060000004E000020032003222A900E3
:10A66000EEFF370032C2BF00614060000004E0002E
:10A67000EAFF320011E1A900B011800080407800AB
:10A680001E007800014878000080FA0000000600F3
:10A690000C00FA0030079800420798005307980012
:10A6A0000000EB00000F78001A003700CE00900089
:10A6B0005E009000A6000700100798002107980090
:10A6C000CE4090003E009000014878003E0090008F
:10A6D0008000E8003E409000804878003E009000F6
:10A6E0008080E8002E409000804878003E00900076
:10A6F00063004000300798004E009000DE0090009C
:10A7000062004000E0804800400798005107980030
:10A710001E0FE800F01F20009E0F1000E3FF340022
:10A720000080FA00000006000600FA0010079800FA
:10A73000210798000000EB00000F780007003700A9
:10A740001E007800800078001E009000008040000D
:10A7500010407800060007001E0FE8002E00900051
:10A760009E0F1000F6FF35000080FA000000060082
:10A770000200FA00004F780033C2BF006140600061
:10A780000004E000FCFF32001E00FB00A011880066
:10A790000080FA00000006001600FA00000F980082
:10A7A000120F9800230F98000000EB00100798008C
:10A7B0000000EB00000F78004D0037001E0078000D
:10A7C000800078000E089000008040001040780063
:10A7D000404798009E0078000E08900000804000DE
:10A7E0000000E80010407800504798009E00780074
:10A7F0000E089000008040000080E80010407800C3
:10A80000604798000040EB00704798001E007800F9
:10A81000630F40002E0090003E0190009E089000C3
:10A820002E0A9000800178000400780044000700A0
:10A830001E089000AE0890007F0160006000B80024
:10A84000030020000200700083807000820120005D
:10A8500003002000820F5000838F580008003A0048
:10A860001E089000AE08900040079800510798001D
:10A870002E009000BE0090006007980071079800BD
:10A880001E0090000000E000100032001E0090004A
:10A890000000E80080007800F003200000806000E5
:10A8A0000000E00009003A006E0090007E01900078
:10A8B000CE0090005E0290008001780004007800D5
:10A8C0001F00070010002400120007001E0890005F
:10A8D000AE08900062004000E0804800100F980031
:10A8E000210F98001E0090000000E800100798005B
:10A8F0009E009000F01F2000808F5000AFFF3400BA
:10A900000080FA00000006009001880081007800B5
:10A9100000000600003B880050052000303B880006
:10A92000A00A2000303B880061E7A800000000007A
:10A930000000000061E7AF00FEFF370000000600E6
:10A94000900188008308BB008288BB0000000600DD
:10A95000900188001100BA009180BA000000060042
:10A960000004040000000000000006003200F800AF
:10A97000023B8800900188008108BB005005200040
:10A98000303B8800A00A2000303B880061E7A80027
:10A99000000000000000000061E7AF00FEFF37008C
:10A9A0003200F90000000600000800000406000064
:10A9B00000000000000000000040DA000000FE007F
:10A9C000FFFFFF00FFFFFF00FFFFFF00FFFFFF0093
:10A9D000FFFFFF00FFFFFF00FFFFFF00FFFFFF0083
:10A9E000FFFFFF00FFFFFF00FFFFFF00FFFFFF0073
:10A9F000FFFFFF00FFFFFF00FFFFFF00FFFFFF0063
:0200000401F009
:10000000FFFF0000FFFF0000FFFF0000F8FF0000FF
:100010007EFF00007FFF0000FDFF0000DFFF00000B
:100020004900000001000000000000000000000086
:00000001FF
